:100000000C94381B0C94641B0C94641B0C94641BA0
:100010000C94641B0C94641B0C94641B0C94641B64
:100020000C94641B0C94641B0C94641B0C94641B54
:100030000C94641B0C94D7340C94641B0C94641BB8
:100040000C94641B0C94641B0C94641B0C94641B34
:100050000C94641B0C94641B0C94641B0C94641B24
:100060000C94641B0C94641B0C94641B0C94641B14
:100070000000000000000000000000000000000080
:100080000000000000000000000000000000000070
:100090000000000000000000000000000000000060
:1000A0000000000000000000000000000000000050
:1000B0000000000000000000000000000000000040
:1000C0000000000000000000000000000000000030
:1000D0000000FFF4F4F40000F4E0E0E00000F4E0DD
:1000E000E0E00000F4E0E0E00000F4E0E0E0000028
:1000F000F4E0E0E00000F4E0E0E00000F4E0E0E044
:10010000F49800000000E09800000000E098000073
:100110000000E09800000000E09800000000E09877
:1001200000000000E09800000000E09800000000DF
:10013000000000FFF4F4000000F4E0E0000000F430
:10014000E0E0000000F4E0E0000000F4E0E0000087
:1001500000F4E0E0000000F4E0E0000000F4E0E083
:10016000F4F4980000FFE0E0980000F4E0E098006C
:1001700000F4E0E0980000F4E0E0980000F4E0E033
:10018000980000F4E0E098000000E0E09800000033
:10019000F4F4F4F4F4F4E0E0E0E0E0E0E0E0E0E0E7
:1001A000E0E0E0E0E0E0E0E0E0E0E0E0E0E0E0E04F
:1001B000E0E0E0E0000000000000000000000000BF
:1001C000F4F4F4F4F4F4E0E0E0E0E0E0E0E0E0E0B7
:1001D000E0E0E0E0E0E0E0E0E0E0E0E0E0E0E0E01F
:1001E000E0E0E0E000000000F4E0000000F4E0E007
:1001F000F4F4F4F4F498E0E0E0E0E098E0E0E0E02B
:10020000E098E0E0E0E0E098E0E0E0E0E098E0E0C6
:10021000E0E0E098E0E0E0E0E098E0E0E0E0E098B6
:1002200000FFF4F4F4F400F4E0E0E0E000F4E0E0D7
:10023000E0E000F4E0E0E0E000F4E0E0E0E000F422
:10024000E0E0E0E000F4E0E0E0E000F4E0E0E0E046
:10025000F4F4F4F4F4F4E0E0E0E0E0E0E0E0E0E026
:10026000E0E0E0E0E0E0E0E0E0E0E0E0E0E0E0E08E
:10027000E0E0E0E0E00000000000E000000000003E
:10028000F4980000FFF4E0980000F4E0E09800002B
:10029000F4E0E0980000F4E0E0980000F4E0E0987A
:1002A0000000F4E000000000F4E000000000F4E0D2
:1002B000F4F4F4F4F4F4E0E0E0E0E0E0E0E0E0E0C6
:1002C000E0E0E0E0E0E0E0E0E0E0E0E0E0E0E0E02E
:1002D000E0E0E0E0E0E0E0E00000E0E0E0E000009E
:1002E000F4F4F4F4F4F4E0E0E0E0E0E0E0E0E0E096
:1002F000E0E0E0E0E0E0E0E0E0E0E0E0E0E0E0E0FE
:10030000E0E0E0E00000000000F40000000000F485
:10031000F4F4F4F40000E0E0E0E09800E0E0E0E075
:100320009800E0E0E0E09800E0E0E0E09800E0E045
:10033000E0E09800E0E0E0E09800E0E0E0E0980035
:10034000F4F4F4F4F4F4E0E0E0E0E0E0E0E0E0E035
:10035000E0E0E0E0E0E0E0E0E0E0E0E0E0E0E0E09D
:10036000E0E0E0E0980000000000980000000000DD
:10037000F4F4F4F4F4F4E0E0E0E0E0E0E0E0E0E005
:10038000E0E0E0E0E0E0E0E0E0E0E0E0E0E0E0E06D
:10039000E0E0E0E000F4E0E0E0E000F4E0E0E0E0F5
:1003A000980000FFF4F4980000F4E0E0980000F4F6
:1003B000E0E0980000F4E0E0980000F4E0E098004D
:1003C0000000F4E098000000F4E09800000000F461
:1003D000F4F4F4000000E0E0E0980000E0E0E098D1
:1003E0000000E0E0E0E09800E0E0E0E0E098E0E03D
:1003F000E0E0E098E0E0E0E0E0E0E0E0E0E0E0E045
:1004000000000000F4F4000000F4E0E0000000F45C
:10041000E0E00000F4E0E0E000F4E0E0E0E000F420
:10042000E0E0E0E098E0E0E0E0E0E0E0E0E0E0E014
:10043000F4F4F4980000E0E0E0980000E0E0E098D8
:100440000000E0E0E0980000E0E0E0980000E0E07C
:1004500098000000E0E098000000E0980000000034
:100460000000F4E0E0E00000F4E0E0E00000F4E090
:10047000E0E00000F4E0E0E00000F4E0E0E0000094
:10048000F4E0E0E00000F4E0E0E00000F4E0E0E0B0
:10049000E09800000000E09800000000E0980000F4
:1004A0000000E09800000000E09800000000E098E4
:1004B00000000000E09800000000E098000000004C
:1004C000000000F4E0E0000000F4E0E0000000F4D0
:1004D000E0E0000000F4E0E0000000F4E0E00000F4
:1004E00000F4E0E0000000F4E0E0000000F4E0E0F0
:1004F000E0E098000000E0E098000000E0E09800F4
:100500000000E0E098000000E0E098000000E0E07B
:1005100098000000E0E098000000E0E09800000093
:1005200000000000000000000000000000000000CB
:10053000000000000000F4F4000000F4E0E000001F
:10054000F4E0E0E000F4E0E0E0E0F4E0E0E0E0E04F
:100550000000F4E0E0E000F4E0E0E0E0F4E0E0E0FF
:10056000E0E0E0E0E0E0E0E0E0E0E0E0E0E0E0E08B
:10057000E0E09898E0E0E0980000E0E098000000FB
:10058000E0E0E0E09800E0E0E0980000E0E09800C3
:100590000000E0980000000098000000000000004B
:1005A000000000000000000000000000000000004B
:1005B00000F4E0E0E0E000F4E0E0E0E000F4E0E09F
:1005C000E0E000F4E0E0E0E000F4E0E0E0E000F48F
:1005D000E0E0E0E000F4E0E0E0E000F4E0E0E0E0B3
:1005E000E00000000000E0F4F4F4F4F4E0E0E0E007
:1005F000E0E0E0E0E0E0E0E0E0E0E0E0E0E0E0E0FB
:10060000E0E0E0E0E0E0E0E0E0E0E000000000004A
:10061000000000000000F4F4F4980000E0E0E0982E
:100620000000E0E0E0980000E0E0E0980000E0E09A
:10063000E0980000E0E0E09800000000000000000A
:1006400000000000F4E000000000F4E00000000002
:10065000F4E000000000F4E000000000F4E000001E
:100660000000F4E000000000F4E000000000F4E00E
:10067000E0E0E0E00000E0E0E0E0F4F4E0E0E0E012
:10068000E0E0E0E0E0E0E0E0E0E0E0E0E0E0E0E06A
:10069000E0E0E0E0E0E0E0E0E0E0E0E0E0E000001A
:1006A0000000000000F4F4F4F4F4F498E0E0E0E07A
:1006B000E0E0E0E0E0E0E0E0E0E0E0E0E0E0E0E03A
:1006C000E0E0E0E0E0E0E0E0E0E00000000000F476
:1006D000E0E0E0E09800E0E0E0E09800E0E0E098B2
:1006E0000000E0E098000000E0E098000000E0E09A
:1006F000E0980000E0E0E0E09800E0E0E0E0980052
:100700009800000000009800000000009800000021
:100710000000980000000000980000000000980011
:100720000000000098000000000098000000000099
:10073000F4E0E0E0E0E000F4E0E0E0E000F4E0E03D
:10074000E0E00000F4E0E0E0000000F4E0E00000A1
:10075000F4E0E0E000F4E0E0E0E000F4E0E0E0E01D
:10076000E0E0E0E0E0E0E0E0E0E0E098E0E0E0E0D1
:10077000E098E0E0E0E09800E0E0E0980000E0E0F1
:10078000E0E09800E0E0E0E0E098E0E0E0E0E09821
:1007900098000000000000000000000000000000C1
:1007A0000000000000000000000000000000000049
:1007B0000000000000000000000000000000000039
:1007C000E09800000000E09800000000E0F4F4F47D
:1007D000F4F4E0E0E0E0E0E0E0E0E0E0E0E0E0E0F1
:1007E000E0E0E0E0E0E0E0E0E0E0E0E0E0E0E0E009
:1007F000000000F4E0E0000000F4E0E0F4F4F4F4C1
:10080000E0E0E0E0E0E0E0E0E0E0E0E0E0E0E0E0E8
:10081000E0E0E0E0E0E0E0E0E0E0E0E0E0E0E0E0D8
:10082000E0E0980000F4E0E0980000F4E0E09800D8
:1008300000F4E0E0980000F4E0E0980000F4E0E06C
:10084000980000F4E0E0980000F4E0E0980000F484
:10085000E0E0E0E0E0E0E0E0E0E0E0E0E0E0E0E098
:10086000E0E0E0E0E0E0E0E0E0E0E0E0E0E0E0E088
:10087000E0E0E0E0E0E0E0E0E0E0E0E0E0E0E0E078
:10088000E0980000000098000000000098F4F4F4E4
:10089000F4F4E0E0E0E0E0E0E0E0E0E0E0E0E0E030
:1008A000E0E0E0E0E0E0E0E0E0E0E0E0E0E0E0E048
:1008B000000000000000000000000000F4F4F4F468
:1008C000F498E0E0E0E0E098E0E0E0E0E098E0E0EC
:1008D000E0E0E098E0E0E0E0E098E0E0E0E0E098F0
:1008E000E00000000000E00000000000E0F4F4F48C
:1008F000F4F4E0E0E0E0E0E0E0E0E0E0E0E0E0E0D0
:10090000E0E0E0E0E0E0E0E0E0E0E0E0E0E0E0E0E7
:10091000000000000000000000000000F4F4F4F407
:10092000F4F4E0E0E0E0E0E0E0E0E0E0E0E0E0E09F
:10093000E0E0E0E0E0E0E0E0E0E0E0E0E0E0E0E0B7
:1009400000000000F4E000000000F4E0F498000073
:10095000F4E0E0980000F4E0E0980000F4E0E098B3
:100960000000F4E0E0980000F4E0E0980000F4E01B
:10097000E0E0E0E00000E0E0E0E00000E0E0E0E0F7
:10098000F4F4E0E0E0E0E0E0E0E0E0E0E0E0E0E03F
:10099000E0E0E0E0E0E0E0E0E0E0E0E0E0E0E0E057
:1009A0000000000000F40000000000F4F4F4F4F48F
:1009B000F498E0E0E0E0E0E0E0E0E0E0E0E0E0E06B
:1009C000E0E0E0E0E0E0E0E0E0E0E0E0E0E0E0E027
:1009D000E0E0E0E09800E0E0E0E09800E0E0E0E067
:1009E0009800E0E0E0E09800E0E0E0E09800E0E07F
:1009F000E0E09800E0E0E0E09800E0E0E09800004F
:100A0000980000000000980000000000F4F4F4F4E6
:100A1000F4F4E0E0E0E0E0E0E0E0E0E0E0E0E0E0AE
:100A2000E0E0E0E0E0E0E0E0E0E0E0E0E0E0E0E0C6
:100A300000F4E0E0E0E000F4E0E0E0E0F4F4E0E026
:100A4000E0E0E0E0E0E0E0E0E0E0E0E0E0E0E0E0A6
:100A5000E0E0E0E0E0E0E0E0E0E0E0E0E0E0E0E096
:100A60009800000000009800000000F498000000CA
:100A7000F4E098000000F4E0980000F4E0E0980052
:100A800000F4E0E0980000F4E0E0980000F4E0E01A
:100A9000F4E0E0E0E0E0E0E0E0E0E0E0E0E0E0E042
:100AA000E0E0E0E0E0E0E098E0E0E0E09800E0E0B6
:100AB000E0980000E0E0E0980000E0E0E09800004E
:100AC000E0E0E0E0E0E0E0E0E0E0E0E098E0E0E06E
:100AD000E0E000F4E0E0E0E00000F4E0E0E000004E
:100AE00000F4E0E0000000F4E0E0000000F4E0E0EA
:100AF000980000000000E09800000000E0E098008E
:100B00000000E0E098000000E0E0E0980000E0E095
:100B1000E0980000E0E0E0980000E0E0E0980000ED
:100B2000C7C7C7C7C7C7C7C7C7C7C7C7C7C7C7C755
:100B3000C7C7C7C7C7C7C7C7C7C7C7C7C7C7C7C745
:100B4000C7C7C7C7C7C7C7C7C7C7C7C7C7C7C7C735
:100B500000000000007C000000007C3F000000005E
:100B60007C3F00000000307C000000000030009757
:100B7000060000F697FF9706F6FF97FF9706F6FF29
:100B80003000000000007C30000000007C300000DD
:100B90000000303000000000300000000000A40021
:100BA00000E2C000F652E2F8E2C0A452E2F8E2C06D
:100BB0000000007C300000007C3F7C3000007C3F67
:100BC0007C300000307C303000000030300000000D
:100BD000000000F600000000F6FF00970600F6FF98
:100BE0000000000000000000000000000000000005
:100BF0000000000000E2C0000000E2F8E2C0A40033
:100C0000E2F8E2C0F652C0E2C0C0A45200C0C00088
:100C100000000000000000007C300000007C3F7CF1
:100C20003000007C3F7C300000307C303000000021
:100C30003030C7F600000000F6FF00000000F6FFAD
:100C40000000000000000000E2C0000000E2F8E246
:100C5000C00000E2F8E2C00000C0E2C0C000A4C7CB
:100C6000C0C00000F65200000000A45200000000C6
:100C70000000000000000000000000E20000000092
:100C800000E2007C300000C07C3F7C3000007C3FF4
:100C90007C3000F6307C3030F6FF00303000F6FF5C
:100CA000E2C000000000F8E2C0000000F8E2C0006E
:100CB0000000E2C0C0000000C0C000000000A400AE
:100CC00000000000F65200000000A452001F1400B3
:100CD0000000000000E200000000E2F80000000058
:100CE000E2F800000000C0E20000000000C0007C4C
:100CF000300000F67C3F7C30F6FF7C3F7C30F6FF16
:100D0000C00000000000E2C000000000E2C00000DF
:100D10000000C0C000000000C00000000000A400EF
:100D2000001F1400F6521F3F1F14A4521F3F1F1430
:100D300000000000E2C0000000E2F8E2000000E273
:100D4000F8E2000000C0E2C000000000C0C00000E7
:100D5000000000F600000000F6FF007C3000F6FF07
:100D6000000000000000C00000000000C000000003
:100D70000000C000001F140000001F3F1F14A4004B
:100D80001F3F1F14F652141F1414A4520014140011
:100D90000000000000000000E2C0000000E2F8E2F5
:100DA000C00000E2F8E2C00000C0E2C0C0000000E5
:100DB000C0C0C7F600000000F6FF00000000F6FF0C
:100DC00000000000000000001F140000001F3F1F73
:100DD0001400001F3F1F140000141F141400A4C7A8
:100DE00014140000F65200000000A452000000009D
:100DF00000000000000000000000001F00000000D4
:100E0000001F00E2C0000014E2F8E2C00000E2F8B7
:100E1000E2C000F6C0E2C0C0F6FF00C0C000F6FFAE
:100E20001F14000000003F1F140000003F1F1400AB
:100E300000001F1414000000141400000000A4009F
:100E400000000000F65200000000A45200970600C7
:100E500000000000001F000000001F3F0000000015
:100E60001F3F00000000141F00000000001400E2FB
:100E7000C00000F6E2F8E2C0F6FFE2F8E2C0F6FFDA
:100E80001400000000001F14000000001F140000E8
:100E90000000141400000000140000000000A40072
:100EA00000970600F65297FF9706A45297FF970601
:100EB000000000001F140000001F3F1F0000001F63
:100EC0003F1F000000141F14000000001414000055
:100ED000000000F600000000F6FF00E2C000F6FF90
:100EE00000000000000014000000000014000000DA
:100EF0000000140000970600000097FF9706A4006A
:100F000097FF9706F65206970606A45200060600BB
:100F100000000000000000001F140000001F3F1F21
:100F20001400001F3F1F140000141F1414000000C1
:100F30001414C7F600000000F6FF00000000F6FFE2
:100F40000000000000000000970600000097FF97D7
:100F500006000097FF970600000697060600A4C744
:100F600006060000F65200000000A4520000000037
:100F700000000000000000000000009700000000DA
:100F80000097001F140000061F3F1F1400001F3FA2
:100F90001F1400F6141F1414F6FF00141400F6FFBB
:100FA000970600000000FF9706000000FF9706006C
:100FB0000000970606000000060600000000A400DE
:100FC00000000000F65200000000A452007C300037
:100FD0000000000000970000000097FF00000000E4
:100FE00097FF000000000697000000000006001FA9
:100FF000140000F61F3F1F14F6FF1F3F1F14F6FFDB
:1010000006000000000097060000000097060000A0
:101010000000060600000000060000000000A4001A
:10102000007C3000F6527C3F7C30A4527C3F7C3008
:1010300000000000970600000097FF97000000974F
:10104000FF9700000006970600000000060600005B
:10105000000000F600000000F6FF001F1400F6FF7D
:101060000000000000000600000000000600000074
:1010700000000600007C300000007C3F7C30A400B3
:101080007C3F7C30F652307C3030A452003030004F
:101090000000000000000000970600000097FF9786
:1010A00006000097FF97060000069706060000005E
:1010B0000606C7F600000000F6FF00000000F6FF7D
:1010C00000000000000000007C300000007C3F7C3D
:1010D0003000007C3F7C300000307C303000A4C702
:1010E00030300000F65200000000A4520000000062
:1010F00000000000000000000000007C0000000074
:10110000007C00970600003097FF9706000097FFCD
:10111000970600F606970606F6FF00060600F6FF9D
:101120007C30000000003F7C300000003F7C30003D
:1011300000007C3030000000303000000000A400CF
:1011400000000000F65200000000A45200E2C000BF
:1011500006970606A4F600060600005200000000EE
:10116000001F000000001F3F000000001F3F0000A4
:101170000000141F00000000001400000000000028
:101180005252C0E2C0C0520000C0C00014000000B3
:1011900000001F14000000001F14000000001414C1
:1011A000000000001400000000000000000000002B
:1011B00097FF9706A4F697FF970600520697060634
:1011C0000000000606000000000000000000000013
:1011D000000000000000000000000000000000000F
:1011E000525200000000520000000000001F1400D6
:1011F00000001F3F1F1400001F3F1F140000141F9A
:10120000141400000014140000000000000000008E
:1012100000000000A4F600009706C7520097FF9751
:1012200006000097FF9706000006970606000000DC
:1012300006060000000000000000000000000000A2
:1012400052520000000052C71F140000001F3F1F31
:101250001400001F3F1F140000141F14140000008E
:101260001414000000000000000000000000000056
:1012700000000000A4F60000000000520000000082
:10128000970600000097FF9700000097FF97000067
:10129000000697060000000006060000000000009F
:1012A00052521F3F1F1452001F3F1F140000141FF3
:1012B00014140600001414000600000000000600CC
:1012C000000000000000000000000000000000001E
:1012D000307C3030A4F600303000005200000000B6
:1012E00000970000000097FF0000000097FF00003B
:1012F000000006970000000000060000000000004B
:101300005252141F1414520000141400060000005E
:101310000000970600000000970600000000060687
:1013200000000000060000000000000000000000B7
:101330007C3F7C30A4F67C3F7C300052307C3030E7
:10134000000000303000009700000000009700000F
:101350000000000600000000000000000000000087
:1013600052520000000052000000000097060000EA
:101370000000FF9706000000FF9706000000970698
:10138000060000000606000000000000000000004B
:1013900000000000A4F600007C30C752007C3F7CB7
:1013A0003000007C3F7C300000307C30300000009A
:1013B00030300000000000000000000000000000CD
:1013C00052520000000052C7970600000097FF9796
:1013D00006000097FF97060000069706060000002B
:1013E00006060000000000000000000000000000F1
:1013F00000000000A4F60000000000520000000001
:101400007C300000007C3F7C0000007C3F7C0000C2
:1014100000307C3000000000303000000000000090
:10142000525297FF9706520097FF970600000697C3
:101430000606300000060600300000000000300004
:10144000000000000000000000000000000000009C
:10145000C0E2C0C0A4F600C0C000005200000000FE
:10146000007C000000007C3F000000007C3F00008A
:101470000000307C00000000003000000000000090
:101480005252069706065200000606003000000081
:1014900000007C30000000007C3000000000303094
:1014A000000000003000000000000000000000000C
:1014B000E2F8E2C0A4F6E2F8E2C00052C0E2C0C026
:1014C000000000C0C000007C00000000007C0000A4
:1014D00000000030000000000000000000000000DC
:1014E0005252000000005200000000007C3000005A
:1014F00000003F7C300000003F7C300000007C306A
:10150000300000003030000000000000000000004B
:1015100000000000A4F60000E2C0C75200E2F8E2BA
:10152000C00000E2F8E2C00000C0E2C0C00000005D
:10153000C0C000000000000000000000000000002B
:1015400052520000000052C77C300000007C3F7CFB
:101550003000007C3F7C300000307C3030000000E8
:10156000303000000000000000000000000000001B
:1015700000000000A4F6000000000052000000007F
:10158000E2C0000000E2F8E2000000E2F8E2000041
:1015900000C0E2C000000000C0C000000000000069
:1015A00052527C3F7C3052007C3F7C300000307CCB
:1015B0003030C00000303000C00000000000C0002B
:1015C000000000000000000000000000000000001B
:1015D000141F1414A4F6001414000052000000009C
:1015E00000E200000000E2F800000000E2F8000065
:1015F0000000C0E20000000000C000000000000089
:101600005252307C3030520000303000C0000000B8
:101610000000E2C000000000E2C000000000C0C006
:1016200000000000C00000000000000000000000FA
:101630001F3F1F14A4F61F3F1F140052141F141441
:1016400000000014140000E20000000000E20000AE
:10165000000000C0000000000000000000000000CA
:10166000525200000000520000000000E2C00000E2
:101670000000F8E2C0000000F8E2C0000000E2C094
:10168000C0000000C0C0000000000000000000001A
:1016900000000000A4F600001F14C752001F3F1FE7
:1016A0001400001F3F1F140000141F14140000003A
:1016B0001414000000000000000000000000000002
:1016C00052520000000052C7E2C0000000E2F8E2FF
:1016D000C00000E2F8E2C00000C0E2C0C0000000AC
:1016E000C0C000000000000000000000000000007A
:1016F00000000000A4F600000000005200000000FE
:101700001F140000001F3F1F0000001F3F1F0000AC
:1017100000141F140000000014140000000000005A
:101720005252E2F8E2C05200E2F8E2C00000C0E229
:10173000C0C0140000C0C00014000000000014006D
:101740000000000000000000000000000000000099
:101750000000000000000000000000000000000089
:101760000000000000000000000000000000000079
:101770000000000000000000000000000000000069
:101780000000FF00000000FFFFFF000000FFFFFF60
:1017900000000000FF0000000000FF00000000004B
:1017A000000000000000FF0000000000000000003A
:1017B000FFFF00FFFF00FFFF00FFFF00FF0000FF33
:1017C0000000000000000000000000000000000019
:1017D0000000000000000000000000000000000009
:1017E00000000000000000FF00FF0000FFFFFFFFFF
:1017F000FF0000FF00FF000000FF00FF0000FFFFF0
:10180000FFFFFF0000FF00FF0000000000000000DD
:1018100000FF0000000000FFFFFF0000FF000000CD
:10182000000000FFFF000000000000FF0000FFFFBD
:10183000FF0000000000FF000000000000000000AA
:10184000FFFF0000FF00FFFF0000FF00000000FF9F
:1018500000000000FF00000000FF00000000FF008B
:1018600000FFFF00FF0000FFFF000000000000007D
:1018700000FF00000000FF00FF000000FF00FF006D
:10188000000000FF00000000FF00FF00FF00FF005D
:1018900000FF000000FFFF00FF000000000000004C
:1018A00000FFFF00000000FFFF00000000FF00003D
:1018B0000000000000000000000000000000000028
:1018C0000000000000000000000000000000000018
:1018D0000000FF00000000FF0000000000FF00000B
:1018E000000000FF0000000000FF0000000000FFFB
:1018F000000000000000FF000000000000000000E9
:1019000000FF000000000000FF0000000000FF00DA
:1019100000000000FF0000000000FF0000000000C9
:10192000FF00000000FF00000000000000000000B9
:1019300000000000000000FF00FF000000FFFFFFAC
:101940000000FFFFFFFFFF0000FFFFFF000000FFA0
:1019500000FF000000000000000000000000000088
:101960000000000000000000FF0000000000FF0079
:101970000000FFFFFFFFFF000000FF00000000006D
:10198000FF00000000000000000000000000000058
:101990000000000000000000000000000000000047
:1019A000000000000000000000000000000000FF38
:1019B000FF00000000FFFF00000000FF000000002B
:1019C0000000000000000000000000000000000017
:1019D0000000FFFFFFFFFF0000000000000000000C
:1019E00000000000000000000000000000000000F7
:1019F00000000000000000000000000000000000E7
:101A0000000000000000000000000000000000FFD7
:101A1000FF00000000FFFF000000000000000000C9
:101A200000000000000000000000FF00000000FFB8
:101A300000000000FF00000000FF00000000FF00A9
:101A40000000000000000000000000000000000096
:101A5000002F2F2F00002F0000002F002F00002F3D
:101A60002F002F002F002F002F2F00002F002F00FE
:101A700000002F00002F2F2F0000000000000000AA
:101A800000002F000000002F2F00000000002F009A
:101A9000000000002F00000000002F0000000000E8
:101AA0002F000000002F2F2F00000000000000007A
:101AB000002F2F2F00002F0000002F00000000003B
:101AC0002F0000002F2F0000002F000000002F002B
:101AD000000000002F2F2F2F2F000000000000001B
:101AE000002F2F2F00002F0000002F00000000000B
:101AF0002F00002F2F2F0000000000002F002F00CC
:101B000000002F00002F2F2F000000000000000019
:101B10000000002F000000002F2F0000002F002FDA
:101B200000002F00002F00002F2F2F2F2F0000006C
:101B3000002F00000000002F000000000000000047
:101B40002F2F2F2F2F002F00000000002F0000004C
:101B500000002F2F2F2F0000000000002F002F006B
:101B600000002F00002F2F2F0000000000000000B9
:101B700000002F2F0000002F000000002F000000A9
:101B800000002F2F2F2F00002F0000002F002F000C
:101B900000002F00002F2F2F000000000000000089
:101BA0002F2F2F2F2F00000000002F000000002FEC
:101BB000000000002F000000002F00000000002F98
:101BC00000000000002F00000000000000000000E6
:101BD000002F2F2F00002F0000002F002F000000EB
:101BE0002F00002F2F2F00002F0000002F002F00AC
:101BF00000002F00002F2F2F000000000000000029
:101C0000002F2F2F00002F0000002F002F000000BA
:101C10002F00002F2F2F2F00000000002F000000AA
:101C2000002F0000002F2F00000000000000000027
:101C300000000000000000000000000000FFFF00A6
:101C4000000000FFFF00000000000000000000FF97
:101C5000FF00000000FFFF00000000000000000087
:101C600000000000000000000000000000FFFF0076
:101C7000000000FFFF00000000000000000000FF67
:101C8000FF00000000FFFF00000000FF0000000058
:101C900000000000FF00000000FF00000000FF0047
:101CA000000000FF000000000000FF000000000036
:101CB00000FF000000000000FF0000000000000026
:101CC000000000000000000000000000FFFFFFFF18
:101CD000FF00000000000000000000000000FFFF07
:101CE000FFFFFF00000000000000000000000000F7
:101CF00000FF000000000000FF000000000000FFE7
:101D0000000000000000FF00000000FF00000000D5
:101D1000FF00000000FF00000000000000000000C5
:101D200000FFFFFF0000FF000000FF0000000000B8
:101D3000FF000000FFFF00000000FF0000000000A7
:101D4000000000000000FF00000000000000000094
:101D500000FFFFFF0000FF000000FF00FF00FFFF8B
:101D6000FF00FF00FF00FF00FF00FFFFFF00FF007C
:101D70000000000000FFFFFF000000000000000066
:101D800000FFFFFF0000FF000000FF00FF00000059
:101D9000FF00FF000000FF00FFFFFFFFFF00FF004C
:101DA0000000FF00FF000000FF0000000000000036
:101DB000FFFFFFFF0000FF000000FF00FF0000002A
:101DC000FF00FFFFFFFF0000FF000000FF00FF001B
:101DD0000000FF00FFFFFFFF000000000000000008
:101DE00000FFFFFF0000FF000000FF00FF000000F9
:101DF0000000FF0000000000FF0000000000FF00E6
:101E00000000FF0000FFFFFF0000000000000000D6
:101E1000FFFFFFFF0000FF000000FF00FF000000C9
:101E2000FF00FF000000FF00FF000000FF00FF00B8
:101E30000000FF00FFFFFFFF0000000000000000A7
:101E4000FFFFFFFFFF00FF0000000000FF00000099
:101E50000000FFFFFFFF0000FF0000000000FF0088
:101E600000000000FFFFFFFFFF0000000000000077
:101E7000FFFFFFFFFF00FF0000000000FF00000069
:101E80000000FFFFFFFF0000FF0000000000FF0058
:101E900000000000FF000000000000000000000043
:101EA00000FFFFFF0000FF000000FF00FF00000038
:101EB0000000FF00FFFFFF00FF000000FF00FF0029
:101EC0000000FF0000FFFFFFFF0000000000000017
:101ED000FF000000FF00FF000000FF00FF00000007
:101EE000FF00FFFFFFFFFF00FF000000FF00FF00FB
:101EF0000000FF00FF000000FF00000000000000E5
:101F000000FFFFFF00000000FF0000000000FF00D6
:101F100000000000FF0000000000FF0000000000C3
:101F2000FF00000000FFFFFF0000000000000000B5
:101F300000000000FF0000000000FF0000000000A3
:101F4000FF0000000000FF00FF000000FF00FF0096
:101F50000000FF0000FFFFFF000000000000000085
:101F6000FF000000FF00FF0000FF0000FF00FF0077
:101F70000000FFFF00000000FF00FF000000FF0066
:101F800000FF0000FF000000FF0000000000000054
:101F9000FF0000000000FF0000000000FF00000044
:101FA0000000FF0000000000FF0000000000FF0034
:101FB00000000000FFFFFFFFFF0000000000000026
:101FC000FF000000FF00FFFF00FFFF00FF00FF0019
:101FD000FF00FF000000FF00FF000000FF00FF0007
:101FE0000000FF00FF000000FF00000000000000F4
:101FF000FF000000FF00FFFF0000FF00FF00FF00E8
:10200000FF00FF0000FFFF00FF000000FF00FF00D7
:102010000000FF00FF000000FF00000000000000C3
:1020200000FFFFFF0000FF000000FF00FF000000B6
:10203000FF00FF000000FF00FF000000FF00FF00A6
:102040000000FF0000FFFFFF000000000000000094
:10205000FFFFFFFF0000FF000000FF00FF00000087
:10206000FF00FFFFFFFF0000FF0000000000FF0077
:1020700000000000FF000000000000000000000061
:1020800000FFFFFF0000FF000000FF00FF00000056
:10209000FF00FF000000FF00FF00FF00FF00FF0047
:1020A00000FF000000FFFF00FF0000000000000034
:1020B000FFFFFFFF0000FF000000FF00FF00000027
:1020C000FF00FFFFFFFF0000FF0000FF0000FF0018
:1020D0000000FF00FF000000FF0000000000000003
:1020E00000FFFFFF0000FF000000FF00FF000000F6
:1020F000000000FFFFFF000000000000FF00FF00E5
:102100000000FF0000FFFFFF0000000000000000D3
:10211000FFFFFFFFFF000000FF0000000000FF00C6
:1021200000000000FF0000000000FF0000000000B1
:10213000FF0000000000FF000000000000000000A1
:10214000FF000000FF00FF000000FF00FF00000094
:10215000FF00FF000000FF00FF000000FF00FF0085
:102160000000FF0000FFFFFF000000000000000073
:10217000FF000000FF00FF000000FF00FF00000064
:10218000FF00FF000000FF00FF000000FF0000FF55
:1021900000FF00000000FF00000000000000000041
:1021A000FF000000FF00FF000000FF00FF00FF0035
:1021B000FF00FF00FF00FF00FF00FF00FF00FF0027
:1021C000FF00FF0000FF00FF000000000000000013
:1021D000FF000000FF00FF000000FF0000FF00FF05
:1021E00000000000FF00000000FF00FF0000FF00F3
:1021F0000000FF00FF000000FF00000000000000E2
:10220000FF000000FF00FF000000FF00FF000000D3
:10221000FF0000FF00FF00000000FF0000000000C2
:10222000FF0000000000FF000000000000000000B0
:10223000FFFFFFFF0000000000FF00000000FF00A4
:10224000000000FF00000000FF0000000000FF0091
:1022500000000000FFFFFFFF000000000000000082
:102260000000FFFF000000FF0000000000FF000072
:102270000000FFFF0000000000FF0000000000FF62
:10228000000000000000FFFF000000000000000050
:102290000000FFFF000000FF0000FF00FF00FFFF45
:1022A00000FFFF00FF0000FFFF00FFFF00FF00FF37
:1022B0000000FF000000FFFF000000000000000021
:1022C00000FFFF000000000000FF0000000000FF12
:1022D0000000000000FFFF00000000FF0000000001
:1022E00000FF000000FFFF000000000000000000F1
:1022F000FEFEFEFEFEFEFEFEFEFEFEFEFEFEFEFEFE
:10230000FEFEFEFEFEFEFEFEFEFEFEFEFEFEFEFEED
:10231000FEFEFEFEFEFEFEFEFEFEFEFEFEFEFEFEDD
:102320005EAFAFAFAFB7A61516161616A6151616E2
:102330001616A61516161616A61516161616A61590
:1023400016161616A61516161616A615161616160F
:102350005C0CAFAFAF560B651E1615090B651E164C
:1023600015090B651E1615090B5C0A1615090B0BD2
:10237000010001550BA5B7AFAE490B651E16150937
:10238000A61516161616A61516161616000B1616F0
:10239000160CB7530016160CA666AE000049A6151B
:1023A00016AFAF52A6151616154A14000000005EAF
:1023B0000B651E1615090B651E161509535F1516BC
:1023C0001509535F151615096715161615096615B3
:1023D000161615096715161609085C000000015548
:1023E000AFAFAFAFAFAF15161616150A1516161606
:1023F000150A00000000000015160A15161615161D
:102400000A15161615160A1516160000000000000B
:10241000AFAFAFAFAFAE16161616150916161616D5
:10242000150900000000000816150A1616551615A5
:102430000A16165516150A16165500000000000853
:1024400015161616150A15161616150A1516161649
:10245000150A00000000000015160A1516161516BC
:102460000A15161615160A151616000000000000AB
:102470001616161615091616161615091616161618
:10248000150900000000000816150A161655161545
:102490000A16165516150A161655000000000008F3
:1024A000FEFE0000FEFEFE005F0400FE005FFF0770
:1024B00004000007070704000006070604000004E4
:1024C00006060400FE00040400FEFEFE0000FEFE00
:1024D000FEFE0000FEFEFE00EA9900FE00EAFFE2BA
:1024E000490000E2E2E249000099E299490000490E
:1024F00099994900FE00494900FEFEFE0000FEFEDB
:10250000FEFE0000FEFEFE007D2100FE007DFF318C
:102510001900003131311900002131211900001951
:1025200021211900FE00191900FEFEFE0000FEFE2A
:10253000FEFE0000FEFEFE00F78600FE00F7FFC76D
:102540004C0000C7C7C74C000086C7864C00004C33
:1025500086864C00FE004C4C00FEFEFE0000FEFE97
:10256000E3E3E3E3E3E3E3E3E3E3E3E3E3E3E3E33B
:10257000E3E3E3E3E3E3E3E3E3E3E3E3E3E3E3E32B
:10258000E3E3E3E3E3E3E3E3E3E3E3E3E3E3E3E31B
:10259000FEFE06FEFEFEFE060706FEFE06079F077F
:1025A00006FE069F070604FE0607060604FEFE0654
:1025B0000604FEFEFEFE04FEFEFEFEFEFEFEFEFE27
:1025C000FEFE30FEFEFEFE303830FEFE30383F3874
:1025D00020FE303F382018FE3038202018FEFE2024
:1025E0002018FEFEFEFE18FEFEFEFEFEFEFEFEFEB5
:1025F000FEFEF0FEFEFEFEF0F8F0FEFEF0F8FBF848
:10260000E0FEF0FBF8E0C8FEF0F8E0E0C8FEFEE017
:10261000E0C8FEFEFEFEC8FEFEFEFEFEFEFEFEFE64
:10262000FEFE37FEFEFEFE373F37FEFE373FFF3F22
:1026300027FE37FF3F271FFE373F27271FFEFE27B6
:10264000271FFEFEFEFE1FFEFEFEFEFEFEFEFEFE3F
:10265000FEFECEFEFEFEFECEDFCEFEFECEDFF7DFBE
:10266000CCFECEF7DFCCC4FECEDFCCCCC4FEFECC9D
:10267000CCC4FEFEFEFEC4FEFEFEFEFEFEFEFEFE20
:10268000FEFE06FEFEFEFE060706FEFE06079F078E
:1026900006FE069F070604FE0607060604FE000661
:1026A000060400FEFE000400FEFEFEFE00FEFEFE2E
:1026B000FEFE30FEFEFEFE303830FEFE30383F3883
:1026C00020FE303F382018FE3038202018FE002031
:1026D000201800FEFE001800FEFEFEFE00FEFEFEBC
:1026E000FEFEF0FEFEFEFEF0F8F0FEFEF0F8FBF857
:1026F000E0FEF0FBF8E0C8FEF0F8E0E0C8FE00E025
:10270000E0C800FEFE00C800FEFEFEFE00FEFEFE6B
:10271000FEFE37FEFEFEFE373F37FEFE373FFF3F31
:1027200027FE37FF3F271FFE373F27271FFE0027C3
:10273000271F00FEFE001F00FEFEFEFE00FEFEFE46
:10274000FEFECEFEFEFEFECEDFCEFEFECEDFF7DFCD
:10275000CCFECEF7DFCCC4FECEDFCCCCC4FE00CCAA
:10276000CCC400FEFE00C400FEFEFEFE00FEFEFE27
:1027700053505249544520454E47494E4520444503
:102780004D4F005C3230303820555A45202D2047BF
:10279000504C2056330020202020535441525420C6
:1027A0003D204F5645524C41590053434F524553DB
:1027B00020474F4553204845524521203A29004D96
:1027C000494C45533A3030302052504D2020202083
:1027D000202020202020002020434C415927532036
:1027E0005343524F4C4C2044454D4F2020205C32E7
:1027F00030303820202020202020202020202020A1
:1028000020202000583A00593A0002010000FF0041
:10281000000102030404050404050404030201008A
:1028200000FF000001020304222324252627282973
:102830002A2B2C2D2E2F3031333435363738393A78
:102840003B3C3D3E3F404142DEDDDCDCDCDCDCDCB1
:10285000DDDEDFE0E1E2E4E5E7E9EBEDEFF1F3F502
:10286000F7F9FBFDFF01020405060708080809093E
:1028700008080807060504030200FFFDFCFAF9F743
:10288000F6F4F3F2F1F0EFEEEEEDEDEDEDEDEDEE51
:10289000EEEFF0F1F2F3F4F6F7F8F9FBFCFDFEFFD2
:1028A00000010203030404050505040404030202F5
:1028B0000100FFFDFCFBFAF8F7F5F4F2F1EFEDECA7
:1028C000EAE9E7E6E4E3E1E0DEDCDBD9D8D6D5D31C
:1028D000D1CFCECCCAC8C6C4C3C1BFBDBBB9B7B5C2
:1028E000B3B1AFADACAAA9A7A6A5A4A3A2A2A1A16A
:1028F000A1A1A2A2A3A4A5A6A7A9ABACAEB0B3B553
:10290000B7BABCBFC2C5C7CACDD0D3D5D8DBDDE00E
:10291000E3E5E8EAECEEF1F3F5F6F8FAFBFDFEFF8D
:102920000001020303040404050504040403030274
:102930000100FFFEFCFBF9F8F6F5F3F1EFEEECEA2F
:10294000E8E7E5E4E2E1E0DF150301020304050640
:102950000708090A0B0C0D0E0F101112131415168F
:102960001718191A1B1C1D1E1F202122232425267F
:102970002728292A2B2C2D2E2F303132333435366F
:102980003738393A3B3C3D3E3F1503020304050608
:102990000708090A060B0C0D0E090F10111213146B
:1029A00015161718191A1B1C1D1E1F2021221C2367
:1029B0001C23242526152728292A2B2C1C2D2E2FB5
:1029C0003031321C33343536373860626567696CB4
:1029D0006E707375777A7C7E80838587898B8D8F07
:1029E00091939597999B9D9FA0A2A4A6A7A9AAACF5
:1029F000ADAEB0B1B2B4B5B6B7B8B9BABABBBCBD7A
:102A0000BDBEBEBFBFBFC0C0C0C0C0C0C0C0C0BFD1
:102A1000BFBFBEBEBDBDBCBBBABAB9B8B7B6B5B410
:102A2000B2B1B0AEADACAAA9A7A6A4A2A09F9D9B2F
:102A300099979593918F8D8B89878583807E7C7AFA
:102A4000777573706E6C69676562605E5B59575429
:102A500052504D4B49464442403D3B393735333166
:102A60002F2D2B2927252321201E1C1A1917161458
:102A70001312100F0E0C0B0A0908070606050403B3
:102A8000030202010101000000000000000000013B
:102A9000010102020303040506060708090A0B0CDC
:102AA0000E0F101213141617191A1C1E202123259D
:102AB00027292B2D2F31333537393B3D40424446B2
:102AC000494B4D50525457595B5E80868C92989E6C
:102AD000A5AAB0B6BCC1C6CBD0D5DADEE2E6EAED37
:102AE000F0F3F5F8FAFBFDFEFEFFFFFFFEFEFDFB37
:102AF000FAF8F5F3F0EDEAE6E2DEDAD5D0CBC6C1BE
:102B0000BCB6B0AAA59E98928C868079736D6761D9
:102B10005A554F49433E39342F2A25211D19151284
:102B20000F0C0A0705040201010000000101020464
:102B300005070A0C0F1215191D21252A2F34393EBD
:102B400043494F555A61676D73797F868C92989E81
:102B5000A5AAB0B6BCC1C6CBD0D5DADEE2E6EAEDB6
:102B6000F0F3F5F8FAFBFDFEFEFFFFFFFEFEFDFBB6
:102B7000FAF8F5F3F0EDEAE6E2DEDAD5D0CBC6C13D
:102B8000BCB6B0AAA59E98928C868079736D676159
:102B90005A554F49433E39342F2A25211D19151204
:102BA0000F0C0A07050402010100000001010204E4
:102BB00005070A0C0F1215191D21252A2F34393E3D
:102BC00043494F555A61676D73791F1D1C1A1917B8
:102BD000151412110F0D0C0A090806050302010055
:102BE000FFFEFCFBFBFAF9F8F7F7F6F6F5F5F5F45E
:102BF000F4F4F4F4F4F4F4F4F5F5F5F6F6F7F7F884
:102C0000F8F9FAFAFBFCFDFDFEFF000001020303E8
:102C10000405060607080809090A0A0A0B0B0B0B2C
:102C20000B0B0B0B0B0B0B0A0A0A0909080706060C
:102C3000050403020100FEFDFCFBF9F8F6F5F3F2D2
:102C4000F0EFEDECEAE8E7E5E4E2E1DFDDDCDBD93B
:102C5000D8D6D5D4D3D1D0CFCECDCDCCCBCBCACA7C
:102C6000C9C9C9C9C8C9C9C9C9CACACBCBCCCDCEC3
:102C7000CFD0D1D3D4D5D7D8DADCDDDFE1E3E5E7B7
:102C8000E9EBEEF0F2F4F6F9FBFD00020407090BA4
:102C90000D10121416181A1C1E2022242527292A6A
:102CA0002B2D2E2F303132333435353636363737FB
:102CB00037373736363635353433333231302F2ED9
:102CC0002D2C2A2928262523222002023A3B5A5B52
:102CD00002023C3D5C5D02023E3F5E5F02024041FB
:102CE000606102024243626302024445646502027B
:102CF0004647666702024849686902024A4B6A6BA6
:102D000002024C4D6C6D02024E4F6E6F020250512A
:102D100070710202525372730202545574750202AA
:102D20005657767702025859787900000000000063
:102D30000000000000000000000000000000000093
:102D40000000000000000000000000000000000083
:102D50000000000000000000000000000000000073
:102D60000000000000000000000000000000000063
:102D7000000000000000000000000000004900000A
:102D800000495252000052525C2D00000000000029
:102D900000000000000000000000004000000049AA
:102DA0004A52004952525B1C52531C25241B2425B5
:102DB000251B0A0A2D1C12120A0A0000000000003E
:102DC0000000404949494949525B5B5B525B1C1C0E
:102DD0001312241C1209090912090909090A0A0A0D
:102DE0000A0A0A13120A0A12130A0000000000005D
:102DF00092525252525213121309001C0A121240DC
:102E00001B65090A0009241B120000251C1C010077
:102E100025241C1C0024252424240000000000007C
:102E20005249494000001B1352494900641C1C5B75
:102E30004A481C651C2552491C1C652464491C1CFD
:102E4000652564491C1C6D2E5C49000000000000D3
:102E50000000000000490000000053520000005331
:102E6000522500004A52252500005B251300005B17
:102E700053000A1C095B1C657F374052522E2E1CE2
:102E8000525C2E251B1324251C1C12002525120024
:102E900000121B0000132E37001B37372E2E37373A
:102EA0002E2E2E2E2E2E6E6E6E1C13131200091354
:102EB0001200001213130012251C13132E371C13BB
:102EC0001313361C131B1B1B25131C1C1B1B1B1C49
:102ED0001C1C1C1C1C1C1C1C1C1313121213130086
:102EE0001313131C000913131C010037131C1300C8
:102EF0002E2E1C1C001C772E2500137F251C010A7A
:102F000037241C1C0A2E25250900132E24252525CF
:102F10002E252525252525252D2E251B2E2E251C48
:102F20001325251C1C1C1C011C1C1300011C0A0061
:102F30000165775C016E7F6E521B25256D1C524921
:102F400025251C1353001C1C1C524A001B135B5BE1
:102F5000000009525C0000005B5C000000001B00E8
:102F600000000000000000000000135B7F776E6E21
:102F7000136577766E6E1B65777676761B5BBF760C
:102F8000B67609136DBFB7B6001B125C76BF0000A2
:102F9000121B125B00000000090A6E6E6E77241C83
:102FA0006E6E77251C1C6E776E1C1C1C76761C1CA6
:102FB0002425B765646D6D1B766D6D5B09125B5CD6
:102FC0005B125B641213131B12121C1C1C1C1C24AE
:102FD0001C1C242525242425251B00002513000066
:102FE00064BF00096EBFBF6D6EBF6D5B12135B12D5
:102FF000131209000901000000002E1C0900096ECF
:10300000010009767F7F12777F7F6412BF775B12A2
:103010001B095B121B0900001B09000000000000D7
:10302000000000000000000000007F7F5313130029
:1030300064121B0100001B120000000000000000D1
:103040000000000000000000000000000000000080
:103050000000000000000000000000000000000070
:103060002600000026002F0000002F00370000007F
:103070003700FF000000FF00BF000000BF00370066
:1030800000370000002626000000000000000000BD
:10309000262626262600000000002F00000000370C
:1030A00000000000FF00000000BF0000000037002B
:1030B0000000000026262626260000000000000052
:1030C0002626262626002F000000000037000000DC
:1030D0000000FFFFFFFF0000BF00000000003700FE
:1030E0000000000026262626260000000000000022
:1030F0002626262600002F0000002F0037000000A3
:103100003700FFFFFFFF0000BF000000BF003700D7
:1031100000003700262626260000000000000000E0
:10312000000026262600002F00002F003700000098
:103130003700FF000000FF00BF000000BF003700A5
:1031400000370000262626000000000000000000D6
:103150002600000026002F0000002F000037003757
:1031600000000000FF00000000BF00BF00003700AB
:1031700000003700260000002600000000000000CC
:10318000000000000000000000000000000000003F
:10319000000000000000000000000000009B000094
:1031A00000529BA400005B9B6D77000000000000B4
:1031B00000000000000000000000005B000000E4D0
:1031C000F6FF099BEDF6FFBFA4ADBFBFBFBF767F83
:1031D0007FB7B7BF7F766EB7B7BF000000000000B3
:1031E00000005BB6F6F6F6FFFFFFFFBFFFFFFFBF75
:1031F000BFAEFFFFFFB7AD65FFFFB7B6AD65FFFF21
:10320000BFB7AE6EFFFFBFB7B7650000000000009C
:10321000F6F6EDEDADA4B66D6D5C526E656565526A
:1032200065765C5C52536E246552526E25255B5266
:10323000772D2525526E6E2D2525000000000000FB
:10324000A49B9B4900006564A49B92006D252564A6
:103250009349656E652E9B5224256D256552252464
:103260006D2D655225256E2E645200000000000071
:1032700000000000004A000000005B9B0000005BB3
:103280005B2D0000525B2E2E00015B2D1C01005CAB
:103290005B014A654A5B1C6E7F77495B9B77776D64
:1032A0005B65776E65656D2D25255C522E251309AE
:1032B00049641C09095C7F7F091C7F7F777F777FCA
:1032C00077777F7F7776777F7F6E656E6EA4B6FFA8
:1032D000655BA4B7BFFF526DBFBFBFFF7FBFBFBF5E
:1032E000BFFFBFBFB7BFFFFF7FB7BFBFFFFF6EB757
:1032F000BFBFFFFF77BFBFBFFFFFFFFFBFBFB75B12
:10330000FFFFBFBFA464FFFFBFADA47FFFFFBFA44B
:10331000BF7FFFBFADBFBFBFFFB6BFBFBF77F7BFA8
:10332000BFBF7777FFBFBFBF64526D7F6E2E2D2D5D
:103330007F766E6E6E2E777777762E1C7F776E2572
:103340001C25776525251C096E6E1C0949255B49DE
:103350004A6E7F645377BF775B5C256E6E255B4A50
:1033600025651C1B5B002524245B53001C1B5B5C38
:1033700000000A5B640000006464000000005C0060
:10338000000000000000000000005B5C7FBF77765B
:103390005C6D7FB777775C6D7FBF77775C64BFBF0D
:1033A000BFBF0A5C6EBFBFBF0065646DBFBF0000DA
:1033B0005B6D646D00000000125B7777777F6E6E47
:1033C00077777F766D7677BF776D6E76BF7F6D6E20
:1033D000767FBF7676BFBF76BFBFBFB664ADADB6F2
:1033E000B6ADBFFF646DADB6AD6477BFBFBFFFFFC5
:1033F00077BFBFBFFFFF7FBFBFBFFFF6BFB7ADF651
:10340000FFFFA4ADFFFFFFFFFFFFFFFFFFFFFFFF79
:10341000FFF6A4005B5200000000BFBFAD5B64BFBD
:10342000B6ADADBFFFBFFFFFFFFFBF64FFFFBFB67D
:10343000765BFFBFBF5B0000FF5C00000000000088
:1034400000000000000000000000BFBF645C5C00E2
:103450006E5C654900006D5B00000000000000002C
:10346000000000000000000000000000000000005C
:103470000000000000000000000006000400000042
:103480000100020003000400050006000700080018
:1034900009000A000B000C000D000E000F001000C8
:1034A00000001100120013001400150016000600A1
:1034B000030000001700180019001A001B001C0070
:1034C0001D001E001F0020002100220023002400F8
:1034D0002500260000000000020800085504085AD4
:1034E0000000F8000990000A1E32050000FFD634E3
:1034F00000000001000200030004000501000101BA
:10350000010201030104010502000201020202039B
:10351000020402050300030103020303030403057D
:103520000400040104020403040404050500050169
:10353000050205030504050506000601060206034B
:10354000060406050700070107020703070407052D
:103550000800080108020803080408050900090119
:1035600009020903090409050A000A010A020A03FB
:103570000A040A050B000B010B020B030B040B05DD
:103580000C000C010C020C030C040C050D000D01C9
:103590000D020D030D040D050E000E010E020E03AB
:1035A0000E040E050F000F010F020F030F040F058D
:1035B0001000100110021003100410051100110179
:1035C000110211031104110512001201120212035B
:1035D000120412051300130113021303130413053D
:1035E0001400140114021403140414051500150129
:1035F000150215031504150516001601160216030B
:1036000016041605170017011702170317041705EC
:1036100018001801180218031804180519001901D8
:1036200019021903190419051A001A011A021A03BA
:103630001A041A051B001B011B021B031B041B059C
:103640001C001C011C021C031C041C051D001D0188
:103650001D021D031D041D051E001E011E021E036A
:103660001E041E051F001F011F021F031F041F054C
:1036700011241FBECFEFD0E1DEBFCDBF14BE88E165
:103680000FB6F89480936000109260000FBE12E0B5
:10369000A0E0B1E0E2E5FCE802C005900D92A23B9B
:1036A000B107D9F71EE0A2EBB2E001C01D92A43130
:1036B000B107E1F70E94AA3E0E9482350E944A3675
:1036C0000E94811B0C9427460C940000CF93DF933B
:1036D00080E00E940F36EC0191FF05C080E00E945F
:1036E0000F36892BD9F76091B3028091B2020E9404
:1036F000073BD093B602C093B50280E0DF91CF9133
:1037000008952F923F924F925F926F927F928F9285
:103710009F92AF92BF92CF92DF92EF92FF920F9360
:103720001F93DF93CF93CDB7DEB7E6970FB6F8942C
:10373000DEBF0FBECDBF8CEF81B980E995E20E945C
:10374000FB3580E790E00E94D0358AE70E947F3504
:103750000E9458351092970280E80E9400366E0150
:103760000894C11CD11CCE01C1969CAB8BAB0E94AE
:10377000514560E170E00E946D45880F991FF60188
:1037800080830E9451456DE070E00E946D45019676
:10379000880F991FF60181830E94514560E170E016
:1037A0000E946D45F601828383E090E0C80ED91E29
:1037B000EBA9FCA9CE16DF06D1F61092F50A08EFA8
:1037C0001AE00E94514565E070E00E946D45F801E5
:1037D00080830D5F1F4FFBE005351F0791F71092A7
:1037E000B3020E94514566E070E00E946D451C01E5
:1037F0000E94514566E070E00E946D452C0100E298
:1038000010E020E230E040E250E060E070E080E074
:1038100090E00E94AC3B77241AAA19AAEE24B1E0EA
:103820008B2E912CA1E0AA2EB12CFAE0FF2ECE0116
:1038300049969EAB8DAB81E090E00E94403D809127
:10384000AD0D9091AE0D01969093AE0D8093AD0DA0
:1038500073949AE0F91699F5E1E0EE1609F47AC14D
:10386000F7E0EF1609F09BC049E859E26DE180E00E
:103870000E94DA3A8E010F5F1F4F2091AD0D3091FB
:10388000AE0D36952795F8018281992787FD909591
:10389000280F391F2F703070A901440F551F420F98
:1038A000531F440F551F4653534D618180810E9421
:1038B000DA3A0D5F1F4F0C151D05F9F602C0FF2007
:1038C00031F58091B3028F5F8093B302883E11F08F
:1038D000FF2465C0F3E0F093970283E80E9400366E
:1038E00049E859E260E280E00E94DA3A00E210E042
:1038F00023E030E046E150E06DE170E080E090E0F0
:103900000E94AC3B1AAA81E089ABEE2403C091E08F
:10391000F91669F48091B3028F5F8093B302E3E0FC
:10392000EE1619F0FF24F3943AC0EE2403C0F2E03F
:10393000FF16C9F4872D90E0FC01E653F54DE491A4
:10394000E093B3028653964DFC0184918093B202BA
:10395000F3E0EF1609F401C184E0E81609F0FFC0B6
:1039600033E0F32E03C093E0F916C9F410929702E6
:1039700080E80E94003649E859E26DE180E00E944B
:10398000DA3A872D90E0FC01E653F54DE491E0939F
:10399000B3028653964DFC0184918093B202FAA93A
:1039A000F13009F048C006EF1AE0B401A501A1E02A
:1039B000B0E0FA01EE0FFF1FE050FF4F80819181D0
:1039C000A89F9001A99F300DB89F300D112494E05D
:1039D000359527959A95E1F7FB01EE0FFF1FEC5403
:1039E000FE4F80819181FC01AE9FC001AF9F900D81
:1039F000BE9F900D112436E0959587953A95E1F795
:103A00008E5BF801808328592183620D731D6A350E
:103A1000710514F06A557040440D551D4A35510525
:103A200014F04A55504011960D5F1F4FA032B1055A
:103A300009F0BFCF0BC0E6EFFAE08FEF808399E18A
:103A4000918333968BE0E335F807B9F70894811C2E
:103A5000911C9AE58916910424F0E6EAFFEF8E0E98
:103A60009F1E0894A11CB11CFAE5AF16B10424F006
:103A700086EA9FEFA80EB91E639498E7691681F451
:103A8000E3940E94514566E070E00E946D451C0180
:103A90000E94514566E070E00E946D452C0166244D
:103AA0008091AD0D80FF50C0E9A9E13009F04CC014
:103AB0008E010F5F1F4F2091AD0D3091AE0D3695E9
:103AC0002795F8018281992787FD9095280F391F46
:103AD0002F703070A901440F551F420F531F440F20
:103AE000551F4653534D618180810E94DA3A0D5F24
:103AF0001F4F8DA99EA908171907E9F68E01075EC9
:103B00001F4FF8012281332727FD30958091AD0D9D
:103B10009091AE0D96958795281B390B2F703070BC
:103B2000A901440F551F420F531F440F551F465301
:103B3000534D618180810E94DA3A0D5F1F4F8BA93E
:103B40009CA908171907E9F60E94661B80E00E94ED
:103B50000F3671CE91E09AAB26CFE1E0EAAB82E07E
:103B6000F82E1DCF163520352E354434141F9122E2
:103B700010268F290F2D9030E8EDC8950000EA95AA
:103B8000E1F7C0ECD2E0002400915E0BC00FD01D25
:103B9000CABDDBBD209120072770022F220F220F04
:103BA000220F70915F0B720F672F262E677026947D
:103BB0002694269410E2219EC00DD11DC0932107AA
:103BC000D0932207EE24A0ECB6E000242011ED01F2
:103BD0002011F72E2011962E201166272011E39434
:103BE00020E8201B00EDA02EA3EBB7E041D000C0E1
:103BF00000C03D01A3E5BBE00EEF14E0ED91FD91A7
:103C00000193019301930193019301931A95B1F7E5
:103C1000D301AA9401F17395639500C0683021F037
:103C200008E00A95F1F7E2CF6627A0960AB41BB424
:103C3000209021073090220723950BF4E1010BF42B
:103C4000692D0BF47F2D0BF4EE2444247030E40432
:103C500009F4E001CBCF05E00A95F1F700000E94DE
:103C60000735E1E0E093620BE2E0E093360008956F
:103C700028980E94ED3E2F931E01C0905B0BD090C0
:103C80005C0B80E323E036E099270D91102F0F7134
:103C9000129516951770C3EFDAE0029FC00DD11D83
:103CA0004880F6010A81089FE00DF11D139FE00D89
:103CB000F11DC3E2D7E0C40DD91FC093530BD093BD
:103CC000540B059009920590099205900992059070
:103CD000099205900992059009920D91102F0F718C
:103CE000129516951770C3EFDAE0029FC00DD11D33
:103CF0004880F6010A81089FE00DF11D139FE00D39
:103D0000F11DC3E2D7E0C40DC093550BD91F289A0B
:103D1000D093560B0590099205900992059009924F
:103D20000590099205900992059009920D91102F26
:103D30000F71129516951770C3EFDAE0029FC00D50
:103D4000D11D4880F6010A81089FE00DF11D139FE7
:103D5000E00DF11DC3E2D7E0C40DD91FC093570B8E
:103D6000D093580B059009920590099205900992FD
:103D70000590099205900992059009920D91102FD6
:103D80000F71129516951770C3EFDAE0029FC00D00
:103D9000D11D4880F6010A81089FE00DF11D139F97
:103DA000E00DF11DC3E2D7E0C40DD91FC093590B3C
:103DB000D0935A0B059009920590099205900992AB
:103DC000059009920590099205900992E101E09110
:103DD000610BEA95E093610B3D01DE013C2F307EE3
:103DE0001EEFC9E2D7E04090640B5090650B26E0CF
:103DF000629FC001ECE6FBE380905D0B40E0E412C3
:103E00008824880C1124E80DF11D05901490F00110
:103E100086944C9120E3429FA395AF71A32B040C91
:103E2000151C080E191E0994F001C895C895C8956F
:103E3000C8950591D990D1120D2D08B94C910591D5
:103E4000D990D1120D2D08B9429F0591D990D11268
:103E50000D2D08B9040C151C0591D990D1120D2D0A
:103E600008B9080E191E0591D990D1120D2D08B967
:103E7000A395AF710591D990D1120D2D08B9A32B3F
:103E8000F0010591D990D1120D2D08B94C910591F1
:103E9000D990D1120D2D08B9429F0591D990D11218
:103EA0000D2D08B9040C151C0591D990D1120D2DBA
:103EB00008B9080E191E0591D990D1120D2D08B917
:103EC000A395AF710591D990D1120D2D08B9A32BEF
:103ED000F0010591D990D1120D2D08B94C910591A1
:103EE000D990D1120D2D08B9429F0591D990D112C8
:103EF0000D2D08B9040C151C0591D990D1120D2D6A
:103F000008B9080E191E0591D990D1120D2D08B9C6
:103F1000A395AF710591D990D1120D2D08B9A32B9E
:103F2000F0010591D990D1120D2D08B94C91059150
:103F3000D990D1120D2D08B9429F0591D990D11277
:103F40000D2D08B9040C151C0591D990D1120D2D19
:103F500008B9080E191E0591D990D1120D2D08B976
:103F6000A395AF710591D990D1120D2D08B9A32B4E
:103F7000F0010591D990D1120D2D08B94C91059100
:103F8000D990D1120D2D08B9429F0591D990D11227
:103F90000D2D08B9040C151C0591D990D1120D2DC9
:103FA00008B9080E191E0591D990D1120D2D08B926
:103FB000A395AF710591D990D1120D2D08B9A32BFE
:103FC000F0010591D990D1120D2D08B94C910591B0
:103FD000D990D1120D2D08B9429F0591D990D112D7
:103FE0000D2D08B9040C151C0591D990D1120D2D79
:103FF00008B9080E191E0591D990D1120D2D08B9D6
:10400000A395AF710591D990D1120D2D08B9A32BAD
:10401000F0010591D990D1120D2D08B94C9105915F
:10402000D990D1120D2D08B9429F0591D990D11286
:104030000D2D08B9040C151C0591D990D1120D2D28
:1040400008B9080E191E0591D990D1120D2D08B985
:10405000A395AF710591D990D1120D2D08B9A32B5D
:10406000F0010591D990D1120D2D08B94C9105910F
:10407000D990D1120D2D08B9429F0591D990D11236
:104080000D2D08B9040C151C0591D990D1120D2DD8
:1040900008B9080E191E0591D990D1120D2D08B935
:1040A000A395AF710591D990D1120D2D08B9A32B0D
:1040B000F0010591D990D1120D2D08B94C910591BF
:1040C000D990D1120D2D08B9429F0591D990D112E6
:1040D0000D2D08B9040C151C0591D990D1120D2D88
:1040E00008B9080E191E0591D990D1120D2D08B9E5
:1040F000A395AF710591D990D1120D2D08B9A32BBD
:10410000F0010591D990D1120D2D08B94C9105916E
:10411000D990D1120D2D08B9429F0591D990D11295
:104120000D2D08B9040C151C0591D990D1120D2D37
:1041300008B9080E191E0591D990D1120D2D08B994
:10414000A395AF710591D990D1120D2D08B9A32B6C
:10415000F0010591D990D1120D2D08B94C9105911E
:10416000D990D1120D2D08B9429F0591D990D11245
:104170000D2D08B9040C151C0591D990D1120D2DE7
:1041800008B9080E191E0591D990D1120D2D08B944
:10419000A395AF710591D990D1120D2D08B9A32B1C
:1041A000F0010591D990D1120D2D08B94C910591CE
:1041B000D990D1120D2D08B9429F0591D990D112F5
:1041C0000D2D08B9040C151C0591D990D1120D2D97
:1041D00008B9080E191E0591D990D1120D2D08B9F4
:1041E000A395AF710591D990D1120D2D08B9A32BCC
:1041F000F0010591D990D1120D2D08B94C9105917E
:10420000D990D1120D2D08B9429F0591D990D112A4
:104210000D2D08B9040C151C0591D990D1120D2D46
:1042200008B9080E191E0591D990D1120D2D08B9A3
:10423000A395AF710591D990D1120D2D08B9A32B7B
:10424000F0010591D990D1120D2D08B94C9105912D
:10425000D990D1120D2D08B9429F0591D990D11254
:104260000D2D08B9040C151C0591D990D1120D2DF6
:1042700008B9080E191E0591D990D1120D2D08B953
:10428000A395AF710591D990D1120D2D08B9A32B2B
:10429000F0010591D990D1120D2D08B94C910591DD
:1042A000D990D1120D2D08B9429F0591D990D11204
:1042B0000D2D08B9040C151C0591D990D1120D2DA6
:1042C00008B9080E191E0591D990D1120D2D08B903
:1042D000A395AF710591D990D1120D2D08B9A32BDB
:1042E000F0010591D990D1120D2D08B94C9105918D
:1042F000D990D1120D2D08B9429F0591D990D112B4
:104300000D2D08B9040C151C0591D990D1120D2D55
:1043100008B9080E191E0591D990D1120D2D08B9B2
:10432000A395AF710591D990D1120D2D08B9A32B8A
:10433000F0010591D990D1120D2D08B94C9105913C
:10434000D990D1120D2D08B9429F0591D990D11263
:104350000D2D08B9040C151C0591D990D1120D2D05
:1043600008B9080E191E0591D990D1120D2D08B962
:10437000A395AF710591D990D1120D2D08B9A32B3A
:10438000F0010591D990D1120D2D08B94C910591EC
:10439000D990D1120D2D08B9429F0591D990D11213
:1043A0000D2D08B9040C151C0591D990D1120D2DB5
:1043B00008B9080E191E0591D990D1120D2D08B912
:1043C000A395AF710591D990D1120D2D08B9A32BEA
:1043D000F0010591D990D1120D2D08B94C9105919C
:1043E000D990D1120D2D08B9429F0591D990D112C3
:1043F0000D2D08B9040C151C0591D990D1120D2D65
:1044000008B9080E191E0591D990D1120D2D08B9C1
:10441000A395AF710591D990D1120D2D08B9A32B99
:10442000F0010591D990D1120D2D08B94C9105914B
:10443000D990D1120D2D08B9429F0591D990D11272
:104440000D2D08B9040C151C0591D990D1120D2D14
:1044500008B9080E191E0591D990D1120D2D08B971
:10446000A395AF710591D990D1120D2D08B9A32B49
:10447000F0010591D990D1120D2D08B94C910591FB
:10448000D990D1120D2D08B9429F0591D990D11222
:104490000D2D08B9040C151C0591D990D1120D2DC4
:1044A00008B9080E191E0591D990D1120D2D08B921
:1044B000A395AF710591D990D1120D2D08B9A32BF9
:1044C000F0010591D990D1120D2D08B94C910591AB
:1044D000D990D1120D2D08B9429F0591D990D112D2
:1044E0000D2D08B9040C151C0591D990D1120D2D74
:1044F00008B9080E191E0591D990D1120D2D08B9D1
:10450000A395AF710591D990D1120D2D08B9A32BA8
:10451000F0012F91000000000027E101D30108B94C
:104520000895F00131964C9100C000C000C000C059
:104530000591D990D1120D2D08B9429F0591D990BE
:10454000D1120D2D08B9040C151C0591D990D1126A
:104550000D2D08B9080E191E0591D990D1120D2DF7
:1045600008B9A395AF710591D990D1120D2D08B955
:10457000A32BF0010591D990D1120D2D08B94C91C2
:104580000591D990D1120D2D08B9429F0591D9906E
:10459000D1120D2D08B9040C151C0591D990D1121A
:1045A0000D2D08B9080E191E0591D990D1120D2DA7
:1045B00008B9A395AF710591D990D1120D2D08B905
:1045C000A32BF0010591D990D1120D2D08B94C9172
:1045D0000591D990D1120D2D08B9429F0591D9901E
:1045E000D1120D2D08B9040C151C0591D990D112CA
:1045F0000D2D08B9080E191E0591D990D1120D2D57
:1046000008B9A395AF710591D990D1120D2D08B9B4
:10461000A32BF0010591D990D1120D2D08B94C9121
:104620000591D990D1120D2D08B9429F0591D990CD
:10463000D1120D2D08B9040C151C0591D990D11279
:104640000D2D08B9080E191E0591D990D1120D2D06
:1046500008B9A395AF710591D990D1120D2D08B964
:10466000A32BF0010591D990D1120D2D08B94C91D1
:104670000591D990D1120D2D08B9429F0591D9907D
:10468000D1120D2D08B9040C151C0591D990D11229
:104690000D2D08B9080E191E0591D990D1120D2DB6
:1046A00008B9A395AF710591D990D1120D2D08B914
:1046B000A32BF0010591D990D1120D2D08B94C9181
:1046C0000591D990D1120D2D08B9429F0591D9902D
:1046D000D1120D2D08B9040C151C0591D990D112D9
:1046E0000D2D08B9080E191E0591D990D1120D2D66
:1046F00008B9A395AF710591D990D1120D2D08B9C4
:10470000A32BF0010591D990D1120D2D08B94C9130
:104710000591D990D1120D2D08B9429F0591D990DC
:10472000D1120D2D08B9040C151C0591D990D11288
:104730000D2D08B9080E191E0591D990D1120D2D15
:1047400008B9A395AF710591D990D1120D2D08B973
:10475000A32BF0010591D990D1120D2D08B94C91E0
:104760000591D990D1120D2D08B9429F0591D9908C
:10477000D1120D2D08B9040C151C0591D990D11238
:104780000D2D08B9080E191E0591D990D1120D2DC5
:1047900008B9A395AF710591D990D1120D2D08B923
:1047A000A32BF0010591D990D1120D2D08B94C9190
:1047B0000591D990D1120D2D08B9429F0591D9903C
:1047C000D1120D2D08B9040C151C0591D990D112E8
:1047D0000D2D08B9080E191E0591D990D1120D2D75
:1047E00008B9A395AF710591D990D1120D2D08B9D3
:1047F000A32BF0010591D990D1120D2D08B94C9140
:104800000591D990D1120D2D08B9429F0591D990EB
:10481000D1120D2D08B9040C151C0591D990D11297
:104820000D2D08B9080E191E0591D990D1120D2D24
:1048300008B9A395AF710591D990D1120D2D08B982
:10484000A32BF0010591D990D1120D2D08B94C91EF
:104850000591D990D1120D2D08B9429F0591D9909B
:10486000D1120D2D08B9040C151C0591D990D11247
:104870000D2D08B9080E191E0591D990D1120D2DD4
:1048800008B9A395AF710591D990D1120D2D08B932
:10489000A32BF0010591D990D1120D2D08B94C919F
:1048A0000591D990D1120D2D08B9429F0591D9904B
:1048B000D1120D2D08B9040C151C0591D990D112F7
:1048C0000D2D08B9080E191E0591D990D1120D2D84
:1048D00008B9A395AF710591D990D1120D2D08B9E2
:1048E000A32BF0010591D990D1120D2D08B94C914F
:1048F0000591D990D1120D2D08B9429F0591D990FB
:10490000D1120D2D08B9040C151C0591D990D112A6
:104910000D2D08B9080E191E0591D990D1120D2D33
:1049200008B9A395AF710591D990D1120D2D08B991
:10493000A32BF0010591D990D1120D2D08B94C91FE
:104940000591D990D1120D2D08B9429F0591D990AA
:10495000D1120D2D08B9040C151C0591D990D11256
:104960000D2D08B9080E191E0591D990D1120D2DE3
:1049700008B9A395AF710591D990D1120D2D08B941
:10498000A32BF0010591D990D1120D2D08B94C91AE
:104990000591D990D1120D2D08B9429F0591D9905A
:1049A000D1120D2D08B9040C151C0591D990D11206
:1049B0000D2D08B9080E191E0591D990D1120D2D93
:1049C00008B9A395AF710591D990D1120D2D08B9F1
:1049D000A32BF0010591D990D1120D2D08B94C915E
:1049E0000591D990D1120D2D08B9429F0591D9900A
:1049F000D1120D2D08B9040C151C0591D990D112B6
:104A00000D2D08B9080E191E0591D990D1120D2D42
:104A100008B9A395AF710591D990D1120D2D08B9A0
:104A2000A32BF0010591D990D1120D2D08B94C910D
:104A30000591D990D1120D2D08B9429F0591D990B9
:104A4000D1120D2D08B9040C151C0591D990D11265
:104A50000D2D08B9080E191E0591D990D1120D2DF2
:104A600008B9A395AF710591D990D1120D2D08B950
:104A7000A32BF0010591D990D1120D2D08B94C91BD
:104A80000591D990D1120D2D08B9429F0591D99069
:104A9000D1120D2D08B9040C151C0591D990D11215
:104AA0000D2D08B9080E191E0591D990D1120D2DA2
:104AB00008B9A395AF710591D990D1120D2D08B900
:104AC000A32BF0010591D990D1120D2D08B94C916D
:104AD0000591D990D1120D2D08B9429F0591D99019
:104AE000D1120D2D08B9040C151C0591D990D112C5
:104AF0000D2D08B9080E191E0591D990D1120D2D52
:104B000008B9A395AF710591D990D1120D2D08B9AF
:104B1000A32BF0010591D990D1120D2D08B94C911C
:104B20000591D990D1120D2D08B9429F0591D990C8
:104B3000D1120D2D08B9040C151C0591D990D11274
:104B40000D2D08B9080E191E0591D990D1120D2D01
:104B500008B9A395AF710591D990D1120D2D08B95F
:104B6000A32BF0010591D990D1120D2D08B94C91CC
:104B70000591D990D1120D2D08B9429F0591D99078
:104B8000D1120D2D08B9040C151C0591D990D11224
:104B90000D2D08B9080E191E0591D990D1120D2DB1
:104BA00008B9A395AF710591D990D1120D2D08B90F
:104BB000A32BF0010591D990D1120D2D08B94C917C
:104BC0000591D990D1120D2D08B9429F0591D99028
:104BD000D1120D2D08B9040C151C0591D990D112D4
:104BE0000D2D08B9080E191E0591D990D1120D2D61
:104BF00008B9A395AF710591D990D1120D2D08B9BF
:104C0000A32BF0010591D990D1120D2D08B94C912B
:104C10002F91000000000027D301E10108B9089599
:104C2000F00132964C91429F00C000C000C0059137
:104C3000D990D1120D2D08B9040C151C0591D990ED
:104C4000D1120D2D08B9080E191E0591D990D11257
:104C50000D2D08B9A395AF710591D990D1120D2DE5
:104C600008B9A32BF0010591D990D1120D2D08B9E7
:104C70004C910591D990D1120D2D08B9429F059103
:104C8000D990D1120D2D08B9040C151C0591D9909D
:104C9000D1120D2D08B9080E191E0591D990D11207
:104CA0000D2D08B9A395AF710591D990D1120D2D95
:104CB00008B9A32BF0010591D990D1120D2D08B997
:104CC0004C910591D990D1120D2D08B9429F0591B3
:104CD000D990D1120D2D08B9040C151C0591D9904D
:104CE000D1120D2D08B9080E191E0591D990D112B7
:104CF0000D2D08B9A395AF710591D990D1120D2D45
:104D000008B9A32BF0010591D990D1120D2D08B946
:104D10004C910591D990D1120D2D08B9429F059162
:104D2000D990D1120D2D08B9040C151C0591D990FC
:104D3000D1120D2D08B9080E191E0591D990D11266
:104D40000D2D08B9A395AF710591D990D1120D2DF4
:104D500008B9A32BF0010591D990D1120D2D08B9F6
:104D60004C910591D990D1120D2D08B9429F059112
:104D7000D990D1120D2D08B9040C151C0591D990AC
:104D8000D1120D2D08B9080E191E0591D990D11216
:104D90000D2D08B9A395AF710591D990D1120D2DA4
:104DA00008B9A32BF0010591D990D1120D2D08B9A6
:104DB0004C910591D990D1120D2D08B9429F0591C2
:104DC000D990D1120D2D08B9040C151C0591D9905C
:104DD000D1120D2D08B9080E191E0591D990D112C6
:104DE0000D2D08B9A395AF710591D990D1120D2D54
:104DF00008B9A32BF0010591D990D1120D2D08B956
:104E00004C910591D990D1120D2D08B9429F059171
:104E1000D990D1120D2D08B9040C151C0591D9900B
:104E2000D1120D2D08B9080E191E0591D990D11275
:104E30000D2D08B9A395AF710591D990D1120D2D03
:104E400008B9A32BF0010591D990D1120D2D08B905
:104E50004C910591D990D1120D2D08B9429F059121
:104E6000D990D1120D2D08B9040C151C0591D990BB
:104E7000D1120D2D08B9080E191E0591D990D11225
:104E80000D2D08B9A395AF710591D990D1120D2DB3
:104E900008B9A32BF0010591D990D1120D2D08B9B5
:104EA0004C910591D990D1120D2D08B9429F0591D1
:104EB000D990D1120D2D08B9040C151C0591D9906B
:104EC000D1120D2D08B9080E191E0591D990D112D5
:104ED0000D2D08B9A395AF710591D990D1120D2D63
:104EE00008B9A32BF0010591D990D1120D2D08B965
:104EF0004C910591D990D1120D2D08B9429F059181
:104F0000D990D1120D2D08B9040C151C0591D9901A
:104F1000D1120D2D08B9080E191E0591D990D11284
:104F20000D2D08B9A395AF710591D990D1120D2D12
:104F300008B9A32BF0010591D990D1120D2D08B914
:104F40004C910591D990D1120D2D08B9429F059130
:104F5000D990D1120D2D08B9040C151C0591D990CA
:104F6000D1120D2D08B9080E191E0591D990D11234
:104F70000D2D08B9A395AF710591D990D1120D2DC2
:104F800008B9A32BF0010591D990D1120D2D08B9C4
:104F90004C910591D990D1120D2D08B9429F0591E0
:104FA000D990D1120D2D08B9040C151C0591D9907A
:104FB000D1120D2D08B9080E191E0591D990D112E4
:104FC0000D2D08B9A395AF710591D990D1120D2D72
:104FD00008B9A32BF0010591D990D1120D2D08B974
:104FE0004C910591D990D1120D2D08B9429F059190
:104FF000D990D1120D2D08B9040C151C0591D9902A
:10500000D1120D2D08B9080E191E0591D990D11293
:105010000D2D08B9A395AF710591D990D1120D2D21
:1050200008B9A32BF0010591D990D1120D2D08B923
:105030004C910591D990D1120D2D08B9429F05913F
:10504000D990D1120D2D08B9040C151C0591D990D9
:10505000D1120D2D08B9080E191E0591D990D11243
:105060000D2D08B9A395AF710591D990D1120D2DD1
:1050700008B9A32BF0010591D990D1120D2D08B9D3
:105080004C910591D990D1120D2D08B9429F0591EF
:10509000D990D1120D2D08B9040C151C0591D99089
:1050A000D1120D2D08B9080E191E0591D990D112F3
:1050B0000D2D08B9A395AF710591D990D1120D2D81
:1050C00008B9A32BF0010591D990D1120D2D08B983
:1050D0004C910591D990D1120D2D08B9429F05919F
:1050E000D990D1120D2D08B9040C151C0591D99039
:1050F000D1120D2D08B9080E191E0591D990D112A3
:105100000D2D08B9A395AF710591D990D1120D2D30
:1051100008B9A32BF0010591D990D1120D2D08B932
:105120004C910591D990D1120D2D08B9429F05914E
:10513000D990D1120D2D08B9040C151C0591D990E8
:10514000D1120D2D08B9080E191E0591D990D11252
:105150000D2D08B9A395AF710591D990D1120D2DE0
:1051600008B9A32BF0010591D990D1120D2D08B9E2
:105170004C910591D990D1120D2D08B9429F0591FE
:10518000D990D1120D2D08B9040C151C0591D99098
:10519000D1120D2D08B9080E191E0591D990D11202
:1051A0000D2D08B9A395AF710591D990D1120D2D90
:1051B00008B9A32BF0010591D990D1120D2D08B992
:1051C0004C910591D990D1120D2D08B9429F0591AE
:1051D000D990D1120D2D08B9040C151C0591D99048
:1051E000D1120D2D08B9080E191E0591D990D112B2
:1051F0000D2D08B9A395AF710591D990D1120D2D40
:1052000008B9A32BF0010591D990D1120D2D08B941
:105210004C910591D990D1120D2D08B9429F05915D
:10522000D990D1120D2D08B9040C151C0591D990F7
:10523000D1120D2D08B9080E191E0591D990D11261
:105240000D2D08B9A395AF710591D990D1120D2DEF
:1052500008B9A32BF0010591D990D1120D2D08B9F1
:105260004C910591D990D1120D2D08B9429F05910D
:10527000D990D1120D2D08B9040C151C0591D990A7
:10528000D1120D2D08B9080E191E0591D990D11211
:105290000D2D08B9A395AF710591D990D1120D2D9F
:1052A00008B9A32BF0010591D990D1120D2D08B9A1
:1052B0004C910591D990D1120D2D08B9429F0591BD
:1052C000D990D1120D2D08B9040C151C0591D99057
:1052D000D1120D2D08B9080E191E0591D990D112C1
:1052E0000D2D08B9A395AF710591D990D1120D2D4F
:1052F00008B9A32BF0010591D990D1120D2D08B951
:105300004C910591D990D1120D2D08B9429F2F9142
:10531000000000000027D301E10108B90895F00161
:1053200033964C91429F040C151C00C000C005919F
:10533000D990D1120D2D08B9080E191E0591D990DA
:10534000D1120D2D08B9A395AF710591D990D11245
:105350000D2D08B9A32BF0010591D990D1120D2D77
:1053600008B94C910591D990D1120D2D08B9429FE1
:105370000591D990D1120D2D08B9040C151C059179
:10538000D990D1120D2D08B9080E191E0591D9908A
:10539000D1120D2D08B9A395AF710591D990D112F5
:1053A0000D2D08B9A32BF0010591D990D1120D2D27
:1053B00008B94C910591D990D1120D2D08B9429F91
:1053C0000591D990D1120D2D08B9040C151C059129
:1053D000D990D1120D2D08B9080E191E0591D9903A
:1053E000D1120D2D08B9A395AF710591D990D112A5
:1053F0000D2D08B9A32BF0010591D990D1120D2DD7
:1054000008B94C910591D990D1120D2D08B9429F40
:105410000591D990D1120D2D08B9040C151C0591D8
:10542000D990D1120D2D08B9080E191E0591D990E9
:10543000D1120D2D08B9A395AF710591D990D11254
:105440000D2D08B9A32BF0010591D990D1120D2D86
:1054500008B94C910591D990D1120D2D08B9429FF0
:105460000591D990D1120D2D08B9040C151C059188
:10547000D990D1120D2D08B9080E191E0591D99099
:10548000D1120D2D08B9A395AF710591D990D11204
:105490000D2D08B9A32BF0010591D990D1120D2D36
:1054A00008B94C910591D990D1120D2D08B9429FA0
:1054B0000591D990D1120D2D08B9040C151C059138
:1054C000D990D1120D2D08B9080E191E0591D99049
:1054D000D1120D2D08B9A395AF710591D990D112B4
:1054E0000D2D08B9A32BF0010591D990D1120D2DE6
:1054F00008B94C910591D990D1120D2D08B9429F50
:105500000591D990D1120D2D08B9040C151C0591E7
:10551000D990D1120D2D08B9080E191E0591D990F8
:10552000D1120D2D08B9A395AF710591D990D11263
:105530000D2D08B9A32BF0010591D990D1120D2D95
:1055400008B94C910591D990D1120D2D08B9429FFF
:105550000591D990D1120D2D08B9040C151C059197
:10556000D990D1120D2D08B9080E191E0591D990A8
:10557000D1120D2D08B9A395AF710591D990D11213
:105580000D2D08B9A32BF0010591D990D1120D2D45
:1055900008B94C910591D990D1120D2D08B9429FAF
:1055A0000591D990D1120D2D08B9040C151C059147
:1055B000D990D1120D2D08B9080E191E0591D99058
:1055C000D1120D2D08B9A395AF710591D990D112C3
:1055D0000D2D08B9A32BF0010591D990D1120D2DF5
:1055E00008B94C910591D990D1120D2D08B9429F5F
:1055F0000591D990D1120D2D08B9040C151C0591F7
:10560000D990D1120D2D08B9080E191E0591D99007
:10561000D1120D2D08B9A395AF710591D990D11272
:105620000D2D08B9A32BF0010591D990D1120D2DA4
:1056300008B94C910591D990D1120D2D08B9429F0E
:105640000591D990D1120D2D08B9040C151C0591A6
:10565000D990D1120D2D08B9080E191E0591D990B7
:10566000D1120D2D08B9A395AF710591D990D11222
:105670000D2D08B9A32BF0010591D990D1120D2D54
:1056800008B94C910591D990D1120D2D08B9429FBE
:105690000591D990D1120D2D08B9040C151C059156
:1056A000D990D1120D2D08B9080E191E0591D99067
:1056B000D1120D2D08B9A395AF710591D990D112D2
:1056C0000D2D08B9A32BF0010591D990D1120D2D04
:1056D00008B94C910591D990D1120D2D08B9429F6E
:1056E0000591D990D1120D2D08B9040C151C059106
:1056F000D990D1120D2D08B9080E191E0591D99017
:10570000D1120D2D08B9A395AF710591D990D11281
:105710000D2D08B9A32BF0010591D990D1120D2DB3
:1057200008B94C910591D990D1120D2D08B9429F1D
:105730000591D990D1120D2D08B9040C151C0591B5
:10574000D990D1120D2D08B9080E191E0591D990C6
:10575000D1120D2D08B9A395AF710591D990D11231
:105760000D2D08B9A32BF0010591D990D1120D2D63
:1057700008B94C910591D990D1120D2D08B9429FCD
:105780000591D990D1120D2D08B9040C151C059165
:10579000D990D1120D2D08B9080E191E0591D99076
:1057A000D1120D2D08B9A395AF710591D990D112E1
:1057B0000D2D08B9A32BF0010591D990D1120D2D13
:1057C00008B94C910591D990D1120D2D08B9429F7D
:1057D0000591D990D1120D2D08B9040C151C059115
:1057E000D990D1120D2D08B9080E191E0591D99026
:1057F000D1120D2D08B9A395AF710591D990D11291
:105800000D2D08B9A32BF0010591D990D1120D2DC2
:1058100008B94C910591D990D1120D2D08B9429F2C
:105820000591D990D1120D2D08B9040C151C0591C4
:10583000D990D1120D2D08B9080E191E0591D990D5
:10584000D1120D2D08B9A395AF710591D990D11240
:105850000D2D08B9A32BF0010591D990D1120D2D72
:1058600008B94C910591D990D1120D2D08B9429FDC
:105870000591D990D1120D2D08B9040C151C059174
:10588000D990D1120D2D08B9080E191E0591D99085
:10589000D1120D2D08B9A395AF710591D990D112F0
:1058A0000D2D08B9A32BF0010591D990D1120D2D22
:1058B00008B94C910591D990D1120D2D08B9429F8C
:1058C0000591D990D1120D2D08B9040C151C059124
:1058D000D990D1120D2D08B9080E191E0591D99035
:1058E000D1120D2D08B9A395AF710591D990D112A0
:1058F0000D2D08B9A32BF0010591D990D1120D2DD2
:1059000008B94C910591D990D1120D2D08B9429F3B
:105910000591D990D1120D2D08B9040C151C0591D3
:10592000D990D1120D2D08B9080E191E0591D990E4
:10593000D1120D2D08B9A395AF710591D990D1124F
:105940000D2D08B9A32BF0010591D990D1120D2D81
:1059500008B94C910591D990D1120D2D08B9429FEB
:105960000591D990D1120D2D08B9040C151C059183
:10597000D990D1120D2D08B9080E191E0591D99094
:10598000D1120D2D08B9A395AF710591D990D112FF
:105990000D2D08B9A32BF0010591D990D1120D2D31
:1059A00008B94C910591D990D1120D2D08B9429F9B
:1059B0000591D990D1120D2D08B9040C151C059133
:1059C000D990D1120D2D08B9080E191E0591D99044
:1059D000D1120D2D08B9A395AF710591D990D112AF
:1059E0000D2D08B9A32BF0010591D990D1120D2DE1
:1059F00008B94C910591D990D1120D2D08B9429F4B
:105A00000591D990D1120D2D08B9040C151C2F91B8
:105A1000000000000027D301E10108B90895F0015A
:105A200034964C91429F040C151C080E191E00C0A0
:105A30000591D990D1120D2D08B9A395AF7105919B
:105A4000D990D1120D2D08B9A32BF0010591D99051
:105A5000D1120D2D08B94C910591D990D1120D2D6F
:105A600008B9429F0591D990D1120D2D08B9040CA7
:105A7000151C0591D990D1120D2D08B9080E191ECB
:105A80000591D990D1120D2D08B9A395AF7105914B
:105A9000D990D1120D2D08B9A32BF0010591D99001
:105AA000D1120D2D08B94C910591D990D1120D2D1F
:105AB00008B9429F0591D990D1120D2D08B9040C57
:105AC000151C0591D990D1120D2D08B9080E191E7B
:105AD0000591D990D1120D2D08B9A395AF710591FB
:105AE000D990D1120D2D08B9A32BF0010591D990B1
:105AF000D1120D2D08B94C910591D990D1120D2DCF
:105B000008B9429F0591D990D1120D2D08B9040C06
:105B1000151C0591D990D1120D2D08B9080E191E2A
:105B20000591D990D1120D2D08B9A395AF710591AA
:105B3000D990D1120D2D08B9A32BF0010591D99060
:105B4000D1120D2D08B94C910591D990D1120D2D7E
:105B500008B9429F0591D990D1120D2D08B9040CB6
:105B6000151C0591D990D1120D2D08B9080E191EDA
:105B70000591D990D1120D2D08B9A395AF7105915A
:105B8000D990D1120D2D08B9A32BF0010591D99010
:105B9000D1120D2D08B94C910591D990D1120D2D2E
:105BA00008B9429F0591D990D1120D2D08B9040C66
:105BB000151C0591D990D1120D2D08B9080E191E8A
:105BC0000591D990D1120D2D08B9A395AF7105910A
:105BD000D990D1120D2D08B9A32BF0010591D990C0
:105BE000D1120D2D08B94C910591D990D1120D2DDE
:105BF00008B9429F0591D990D1120D2D08B9040C16
:105C0000151C0591D990D1120D2D08B9080E191E39
:105C10000591D990D1120D2D08B9A395AF710591B9
:105C2000D990D1120D2D08B9A32BF0010591D9906F
:105C3000D1120D2D08B94C910591D990D1120D2D8D
:105C400008B9429F0591D990D1120D2D08B9040CC5
:105C5000151C0591D990D1120D2D08B9080E191EE9
:105C60000591D990D1120D2D08B9A395AF71059169
:105C7000D990D1120D2D08B9A32BF0010591D9901F
:105C8000D1120D2D08B94C910591D990D1120D2D3D
:105C900008B9429F0591D990D1120D2D08B9040C75
:105CA000151C0591D990D1120D2D08B9080E191E99
:105CB0000591D990D1120D2D08B9A395AF71059119
:105CC000D990D1120D2D08B9A32BF0010591D990CF
:105CD000D1120D2D08B94C910591D990D1120D2DED
:105CE00008B9429F0591D990D1120D2D08B9040C25
:105CF000151C0591D990D1120D2D08B9080E191E49
:105D00000591D990D1120D2D08B9A395AF710591C8
:105D1000D990D1120D2D08B9A32BF0010591D9907E
:105D2000D1120D2D08B94C910591D990D1120D2D9C
:105D300008B9429F0591D990D1120D2D08B9040CD4
:105D4000151C0591D990D1120D2D08B9080E191EF8
:105D50000591D990D1120D2D08B9A395AF71059178
:105D6000D990D1120D2D08B9A32BF0010591D9902E
:105D7000D1120D2D08B94C910591D990D1120D2D4C
:105D800008B9429F0591D990D1120D2D08B9040C84
:105D9000151C0591D990D1120D2D08B9080E191EA8
:105DA0000591D990D1120D2D08B9A395AF71059128
:105DB000D990D1120D2D08B9A32BF0010591D990DE
:105DC000D1120D2D08B94C910591D990D1120D2DFC
:105DD00008B9429F0591D990D1120D2D08B9040C34
:105DE000151C0591D990D1120D2D08B9080E191E58
:105DF0000591D990D1120D2D08B9A395AF710591D8
:105E0000D990D1120D2D08B9A32BF0010591D9908D
:105E1000D1120D2D08B94C910591D990D1120D2DAB
:105E200008B9429F0591D990D1120D2D08B9040CE3
:105E3000151C0591D990D1120D2D08B9080E191E07
:105E40000591D990D1120D2D08B9A395AF71059187
:105E5000D990D1120D2D08B9A32BF0010591D9903D
:105E6000D1120D2D08B94C910591D990D1120D2D5B
:105E700008B9429F0591D990D1120D2D08B9040C93
:105E8000151C0591D990D1120D2D08B9080E191EB7
:105E90000591D990D1120D2D08B9A395AF71059137
:105EA000D990D1120D2D08B9A32BF0010591D990ED
:105EB000D1120D2D08B94C910591D990D1120D2D0B
:105EC00008B9429F0591D990D1120D2D08B9040C43
:105ED000151C0591D990D1120D2D08B9080E191E67
:105EE0000591D990D1120D2D08B9A395AF710591E7
:105EF000D990D1120D2D08B9A32BF0010591D9909D
:105F0000D1120D2D08B94C910591D990D1120D2DBA
:105F100008B9429F0591D990D1120D2D08B9040CF2
:105F2000151C0591D990D1120D2D08B9080E191E16
:105F30000591D990D1120D2D08B9A395AF71059196
:105F4000D990D1120D2D08B9A32BF0010591D9904C
:105F5000D1120D2D08B94C910591D990D1120D2D6A
:105F600008B9429F0591D990D1120D2D08B9040CA2
:105F7000151C0591D990D1120D2D08B9080E191EC6
:105F80000591D990D1120D2D08B9A395AF71059146
:105F9000D990D1120D2D08B9A32BF0010591D990FC
:105FA000D1120D2D08B94C910591D990D1120D2D1A
:105FB00008B9429F0591D990D1120D2D08B9040C52
:105FC000151C0591D990D1120D2D08B9080E191E76
:105FD0000591D990D1120D2D08B9A395AF710591F6
:105FE000D990D1120D2D08B9A32BF0010591D990AC
:105FF000D1120D2D08B94C910591D990D1120D2DCA
:1060000008B9429F0591D990D1120D2D08B9040C01
:10601000151C0591D990D1120D2D08B9080E191E25
:106020000591D990D1120D2D08B9A395AF710591A5
:10603000D990D1120D2D08B9A32BF0010591D9905B
:10604000D1120D2D08B94C910591D990D1120D2D79
:1060500008B9429F0591D990D1120D2D08B9040CB1
:10606000151C0591D990D1120D2D08B9080E191ED5
:106070000591D990D1120D2D08B9A395AF71059155
:10608000D990D1120D2D08B9A32BF0010591D9900B
:10609000D1120D2D08B94C910591D990D1120D2D29
:1060A00008B9429F0591D990D1120D2D08B9040C61
:1060B000151C0591D990D1120D2D08B9080E191E85
:1060C0000591D990D1120D2D08B9A395AF71059105
:1060D000D990D1120D2D08B9A32BF0010591D990BB
:1060E000D1120D2D08B94C910591D990D1120D2DD9
:1060F00008B9429F0591D990D1120D2D08B9040C11
:10610000151C0591D990D1120D2D08B9080E191E34
:106110002F91000000000027D301E10108B9089584
:10612000F00135964C91429F040C151C080E191E67
:10613000A395AF710591D990D1120D2D08B9A32B5C
:10614000F0010591D990D1120D2D08B94C9105910E
:10615000D990D1120D2D08B9429F0591D990D11235
:106160000D2D08B9040C151C0591D990D1120D2DD7
:1061700008B9080E191E0591D990D1120D2D08B934
:10618000A395AF710591D990D1120D2D08B9A32B0C
:10619000F0010591D990D1120D2D08B94C910591BE
:1061A000D990D1120D2D08B9429F0591D990D112E5
:1061B0000D2D08B9040C151C0591D990D1120D2D87
:1061C00008B9080E191E0591D990D1120D2D08B9E4
:1061D000A395AF710591D990D1120D2D08B9A32BBC
:1061E000F0010591D990D1120D2D08B94C9105916E
:1061F000D990D1120D2D08B9429F0591D990D11295
:106200000D2D08B9040C151C0591D990D1120D2D36
:1062100008B9080E191E0591D990D1120D2D08B993
:10622000A395AF710591D990D1120D2D08B9A32B6B
:10623000F0010591D990D1120D2D08B94C9105911D
:10624000D990D1120D2D08B9429F0591D990D11244
:106250000D2D08B9040C151C0591D990D1120D2DE6
:1062600008B9080E191E0591D990D1120D2D08B943
:10627000A395AF710591D990D1120D2D08B9A32B1B
:10628000F0010591D990D1120D2D08B94C910591CD
:10629000D990D1120D2D08B9429F0591D990D112F4
:1062A0000D2D08B9040C151C0591D990D1120D2D96
:1062B00008B9080E191E0591D990D1120D2D08B9F3
:1062C000A395AF710591D990D1120D2D08B9A32BCB
:1062D000F0010591D990D1120D2D08B94C9105917D
:1062E000D990D1120D2D08B9429F0591D990D112A4
:1062F0000D2D08B9040C151C0591D990D1120D2D46
:1063000008B9080E191E0591D990D1120D2D08B9A2
:10631000A395AF710591D990D1120D2D08B9A32B7A
:10632000F0010591D990D1120D2D08B94C9105912C
:10633000D990D1120D2D08B9429F0591D990D11253
:106340000D2D08B9040C151C0591D990D1120D2DF5
:1063500008B9080E191E0591D990D1120D2D08B952
:10636000A395AF710591D990D1120D2D08B9A32B2A
:10637000F0010591D990D1120D2D08B94C910591DC
:10638000D990D1120D2D08B9429F0591D990D11203
:106390000D2D08B9040C151C0591D990D1120D2DA5
:1063A00008B9080E191E0591D990D1120D2D08B902
:1063B000A395AF710591D990D1120D2D08B9A32BDA
:1063C000F0010591D990D1120D2D08B94C9105918C
:1063D000D990D1120D2D08B9429F0591D990D112B3
:1063E0000D2D08B9040C151C0591D990D1120D2D55
:1063F00008B9080E191E0591D990D1120D2D08B9B2
:10640000A395AF710591D990D1120D2D08B9A32B89
:10641000F0010591D990D1120D2D08B94C9105913B
:10642000D990D1120D2D08B9429F0591D990D11262
:106430000D2D08B9040C151C0591D990D1120D2D04
:1064400008B9080E191E0591D990D1120D2D08B961
:10645000A395AF710591D990D1120D2D08B9A32B39
:10646000F0010591D990D1120D2D08B94C910591EB
:10647000D990D1120D2D08B9429F0591D990D11212
:106480000D2D08B9040C151C0591D990D1120D2DB4
:1064900008B9080E191E0591D990D1120D2D08B911
:1064A000A395AF710591D990D1120D2D08B9A32BE9
:1064B000F0010591D990D1120D2D08B94C9105919B
:1064C000D990D1120D2D08B9429F0591D990D112C2
:1064D0000D2D08B9040C151C0591D990D1120D2D64
:1064E00008B9080E191E0591D990D1120D2D08B9C1
:1064F000A395AF710591D990D1120D2D08B9A32B99
:10650000F0010591D990D1120D2D08B94C9105914A
:10651000D990D1120D2D08B9429F0591D990D11271
:106520000D2D08B9040C151C0591D990D1120D2D13
:1065300008B9080E191E0591D990D1120D2D08B970
:10654000A395AF710591D990D1120D2D08B9A32B48
:10655000F0010591D990D1120D2D08B94C910591FA
:10656000D990D1120D2D08B9429F0591D990D11221
:106570000D2D08B9040C151C0591D990D1120D2DC3
:1065800008B9080E191E0591D990D1120D2D08B920
:10659000A395AF710591D990D1120D2D08B9A32BF8
:1065A000F0010591D990D1120D2D08B94C910591AA
:1065B000D990D1120D2D08B9429F0591D990D112D1
:1065C0000D2D08B9040C151C0591D990D1120D2D73
:1065D00008B9080E191E0591D990D1120D2D08B9D0
:1065E000A395AF710591D990D1120D2D08B9A32BA8
:1065F000F0010591D990D1120D2D08B94C9105915A
:10660000D990D1120D2D08B9429F0591D990D11280
:106610000D2D08B9040C151C0591D990D1120D2D22
:1066200008B9080E191E0591D990D1120D2D08B97F
:10663000A395AF710591D990D1120D2D08B9A32B57
:10664000F0010591D990D1120D2D08B94C91059109
:10665000D990D1120D2D08B9429F0591D990D11230
:106660000D2D08B9040C151C0591D990D1120D2DD2
:1066700008B9080E191E0591D990D1120D2D08B92F
:10668000A395AF710591D990D1120D2D08B9A32B07
:10669000F0010591D990D1120D2D08B94C910591B9
:1066A000D990D1120D2D08B9429F0591D990D112E0
:1066B0000D2D08B9040C151C0591D990D1120D2D82
:1066C00008B9080E191E0591D990D1120D2D08B9DF
:1066D000A395AF710591D990D1120D2D08B9A32BB7
:1066E000F0010591D990D1120D2D08B94C91059169
:1066F000D990D1120D2D08B9429F0591D990D11290
:106700000D2D08B9040C151C0591D990D1120D2D31
:1067100008B9080E191E0591D990D1120D2D08B98E
:10672000A395AF710591D990D1120D2D08B9A32B66
:10673000F0010591D990D1120D2D08B94C91059118
:10674000D990D1120D2D08B9429F0591D990D1123F
:106750000D2D08B9040C151C0591D990D1120D2DE1
:1067600008B9080E191E0591D990D1120D2D08B93E
:10677000A395AF710591D990D1120D2D08B9A32B16
:10678000F0010591D990D1120D2D08B94C910591C8
:10679000D990D1120D2D08B9429F0591D990D112EF
:1067A0000D2D08B9040C151C0591D990D1120D2D91
:1067B00008B9080E191E0591D990D1120D2D08B9EE
:1067C000A395AF710591D990D1120D2D08B9A32BC6
:1067D000F0010591D990D1120D2D08B94C91059178
:1067E000D990D1120D2D08B9429F0591D990D1129F
:1067F0000D2D08B9040C151C0591D990D1120D2D41
:1068000008B9080E191E0591D990D1120D2D08B99D
:10681000A395AF712F91000000000027D301E10183
:1068200008B90895CC03CC03CC03CC03CC03CC0330
:10683000CC03CC03CC03CC03CC03CC03CC03CC03E0
:10684000CC03CC03CC03CC03CC03CC03CC03CC03D0
:10685000CC03CC03CC03CC03CC03CC03CC03CC03C0
:10686000CC03CC03CC03CC03CC03CC03CC03CC03B0
:10687000CC03CC03CC03CC03CC03CC03CC03CC03A0
:10688000CC03CC03CC03CC0328980E94013FE7E162
:10689000EA95F1F7289A05D1E0E0F6E0E8D0E0FFCC
:1068A00043D0E0FF02C00E94C73D0895129A0C94A5
:1068B00059340C945B341298442755276627772760
:1068C0008CE00C9463340C9465340C9467340C9411
:1068D00069340C946B340C946D34440F551F00993B
:1068E0004160660F771F01996160139A0C947834A8
:1068F0000C947A3413980C947D340C947F340C945B
:1069000081340C9483348A9541F740955095609575
:1069100070955F707F7040936B0B50936C0B60931E
:106920006D0B70936E0B0895EF93E091610BE43E55
:10693000E0F5E431D0F12F923F924F925F926F9247
:106940007F928F929F92AF92BF92CF92DF92EF92FF
:10695000FF920F931F932F933F934F935F936F93E8
:106960007F938F939F93AF93BF93CF93DF930E94B7
:10697000BC1DDF91CF91BF91AF919F918F917F917E
:106980006F915F914F913F912F911F910F91FF90C8
:10699000EF90DF90CF90BF90AF909F908F907F90BF
:1069A0006F905F904F903F902F90EF910895FF93DD
:1069B000EF93EFB7EF93E0918400EE50E13000F0F9
:1069C000E23000F0E33000F0E43000F0E53000F0B9
:1069D000E63000F0E73000F0E83000F0E93000F099
:1069E00005D0EF91EFBFEF91FF9118950F921F9295
:1069F000E4E6FBE30090600B000C1124E00DF11DB8
:106A000005901490F00109951F900F900895289813
:106A10000E94013FE5E1EA95F1F7E091610BEA950B
:106A2000E093610B289A00000000089528980E94C6
:106A30002A3F289A0000E1E0F6E019D02BD0089513
:106A400028980E942A3FE0EB0000EA95E9F7000051
:106A50000000289AF6E0E2E00AD0089528980E9403
:106A60002A3F289A0000E3E0FCEF01D0089500904F
:106A7000610B0A9410905F0011FC0F2E0092610BC5
:106A80000090600B11FC0E2E0092600BE0E011FCF8
:106A9000E1E00895E3E0E0938900EDE8E093880009
:106AA0000895E7E0E0938900EBE1E0938800089522
:106AB000E0E6F4E0A0ECB2E066276D933197E9F7E9
:106AC000112408959927772720E2629F080E191E46
:106AD000A0ECB2E0A00DB11D4C93112408950895CF
:106AE000992720E2629F080E191EA0ECB2E0A00DCB
:106AF000B11D50916A0B450F4C931124089580935A
:106B00006A0B0895F8944427409381004093450010
:106B10004FEF47B944B940E84AB941E04C7F4C6077
:106B200041B91298139800E00093600B06E00093BF
:106B3000610B409385004093840043E040938900BB
:106B40004DE84093880049E04093810042E0409343
:106B50006F0042E44093440040E04093470041E02E
:106B600000004093450043E84093B00040E040936C
:106B7000B30041E04093B10041E045B9789411245D
:106B800040E9A3E2B7E00EEF0D934A95E9F740E044
:106B90004093200708958093680B9093690B0895A4
:106BA0008093640B9093650B08958093660B90938C
:106BB000670B08958091620B089511241092620B67
:106BC0000895882329F480916B0B90916C0B0895A4
:106BD00080916D0B90916E0B089580E891E0809309
:106BE000610090936100089580E890E080936100D7
:106BF00090936100089580935B0B90935C0B0895D4
:106C000080932007089528E088E190E00FB6F8947B
:106C1000A895809360000FBE20936000089588239C
:106C200029F480916B0B90916C0B04C080916D0BDB
:106C300090916E0B9093810B8093800B4091800B11
:106C40005091810B4F3F510519F1CA01807093702B
:106C500080509340E9F4CA01887098708850984039
:106C6000B9F480916B0B90916C0B892B31F0809172
:106C70006D0B90916E0B892BA1F728E088E190E0D5
:106C80000FB6F894A895809360000FBE2093600023
:106C9000CA0108950F931F938EEE94E30E94E3368A
:106CA0000AE21DE2C8010E94D035C8010E94CB351E
:106CB0000E9458358FE090E00E94403D41E06FEF28
:106CC00080E00E942D3A0AE714E3A8016CE088E016
:106CD0000E94F33C83E090E00E94403D4EEA54E382
:106CE0006CE088E00E94F33C82E090E00E94403D2E
:106CF000A8016CE088E00E94F33C88E290E00E94EA
:106D0000403D0E94583584E190E00E94403D1F9133
:106D10000F91089590E025E130E0829FF001839F7C
:106D2000F00D929FF00D1124EF54F24F61870895FA
:106D30006093A80D089590E025E130E0829FF00176
:106D4000839FF00D929FF00D1124EF54F24F1286A5
:106D50001182089590E025E130E0829FF001839F49
:106D6000F00D929FF00D1124EF54F24F81E0828BD1
:106D7000089590E025E130E0829FF001839FF00DBF
:106D8000929FF00D1124EF54F24F6087089590E028
:106D900025E130E0829FF001839FF00D929FF00D7E
:106DA0001124EF54F24F6483089590E025E130E020
:106DB000829FF001839FF00D929FF00D1124EF54FC
:106DC000F24F658308959093080E8093070E1092FA
:106DD000820BE1EBFDE021E08FEF98E12083178249
:106DE0008683138680871182958375963EE0E53011
:106DF000F307A1F708951092B20D1092C70D1092EB
:106E0000DC0D1092F10D01969093100E80930F0EF1
:106E10009093B00D8093AF0D9093130E8093120E4C
:106E200010920E0E10920D0E1092060E1092050E7C
:106E30001092090E81E08093820B10920C0E10923A
:106E40000B0E08958091AF0D9091B00D0E94FB360E
:106E500008958091BA0D87FD03C08AEF8093BA0D23
:106E60008091CF0D87FD03C08AEF8093CF0D809175
:106E7000E40D87FD03C08AEF8093E40D8091F90D46
:106E800087FD03C08AEF8093F90D1092820B08955D
:106E900081E08093820B0895DC01ED91FC911197C4
:106EA000AF014F5F5F4F11965C934E93E4912E2F8D
:106EB00030E0E7FF13C02F7730703695322F22274E
:106EC00037952795FA014F5F5F4FE4918E2F8F77AB
:106ED000280F311DE7FDF1CF4D935C93C901089553
:106EE00008950F931F93CF93DF93182F062FEA0176
:106EF000833049F481E091E09093AA0D8093A90D2D
:106F00002093A80D10C0622F0E949F3D812F90E01A
:106F1000FC01EE0FFF1FE80FF91FEE0FFF1FEB56EE
:106F2000F24FD283C183212F30E085E190E0289F8A
:106F3000F001299FF00D389FF00D1124EF54F24F0E
:106F400081E082870783DF91CF911F910F91089590
:106F50000E949F3D0895EF92FF920F931F93CF934E
:106F6000DF93182F062FF42EE22EC82FD0E085E1F4
:106F700090E0C89FF001C99FF00DD89FF00D11243B
:106F8000EF54F24F8285882321F08181882309F014
:106F900077C0EE2091F485E190E0C89FF001C99F91
:106FA000F00DD89FF00D1124EF54F24F128A818515
:106FB000882309F065C0178263C0133059F481E05B
:106FC00091E09093AA0D8093A90D81E08093A80D84
:106FD0000F2D08C060E0812F0E949F3D6F2D812FF3
:106FE0000E94803D0F3799F485E190E0C89FF00141
:106FF000C99FF00DD89FF00D1124EF54F24F8091EE
:107000000B0E86878CE09EE0948B838B20C0802FB4
:1070100090E0880F991FE091070EF091080EE80F9D
:10702000F91F259134912F5F3F4FF901449185E17C
:1070300090E0C89FF001C99FF00DD89FF00D11247A
:10704000EF54F24F46872F5F3F4F348B238B85E100
:1070500090E0C89FF001C99FF00DD89FF00D11245A
:10706000EF54F24F17861186038711828FEF8087C6
:10707000E782F282108A81E08287128A118A148262
:10708000DF91CF911F910F91FF90EF900895CF92D4
:10709000DF92FF920F931F93CF93DF93E9EBFDE015
:1070A0008181282F332727FD30958081280F311DBE
:1070B0002F3F310519F014F02FEF30E0C90137FFF1
:1070C00002C080E090E0808375964EE0ED30F407DA
:1070D00039F78091820B882309F0D9C0F5C0E0917F
:1070E0000F0EF091100E9F012F5F3F4F3093100E47
:1070F00020930F0E44914F3F69F5A9014F5F5F4FF9
:107100005093100E40930F0EF90184918F3219F4B1
:107110001092820BCAC0863009F0AAC0FA013196DB
:10712000CF0101969093100E80930F0EE491E335FA
:1071300029F49093130E8093120E9AC0E53409F04F
:1071400097C08091120E9091130E9093100E809321
:107150000F0E8EC047FF02C04093090E542F5F7080
:10716000842F90E0807F9070803B910529F1803CD6
:10717000910529F18039910509F038C0C9010196BE
:10718000F901449101969093100E80930F0E019790
:10719000FC012491852F90E08C9FF0018D9FF00DD4
:1071A0009C9FF00D1124EF54F24F8081882309F445
:1071B0005FC0220F638545C02E5F3F4F48C02F5FE1
:1071C0003F4F3093100E20930F0E21503040F901A5
:1071D0002491852F90E08C9FF0018D9FF00D9C9F56
:1071E000F00D1124EF54F24F238742C08091090E15
:1071F000582F5F7090E0807F9070803B910529F15F
:10720000803C910549F18039910591F52F5F3F4F01
:107210003093100E20930F0E21503040F90124912D
:10722000852F90E08C9FD0018D9FB00D9C9FB00D5D
:107230001124AF54B24F8C918823D1F0220F1B96AA
:107240006C91852F0E94AB3713C02F5F3F4F309357
:10725000100E20930F0E0CC0852F90E08C9FF00134
:107260008D9FF00D9C9FF00D1124EF54F24F43873A
:107270008FE09EE00E944C379695879590930E0E76
:1072800080930D0E1092060E1092050E02C0C5E1FD
:10729000D0E06091050E7091060E80910D0E9091D8
:1072A0000E0E6817790709F41ACF6F5F7F4F70933E
:1072B000060E6093050E80910B0E90910C0E0196B8
:1072C00090930C0E80930B0E05E91DE0C2EBDDE000
:1072D000FF248FEFC82ED12C8989882309F05EC046
:1072E0008A899B89892B09F456C09E858D859817BC
:1072F00008F04CC050C08A852A893B898F37E9F451
:10730000D9018D91BB8BAA8B8F3F01F1F90161816E
:107310001196BB8BAA8BE82FF0E0EE0FFF1FE8560B
:10732000FD4F0190F081E02D8F2D0995EA89FB89B1
:1073300081918D87FB8BEA8B28C0A9014F5F5F4F3E
:107340005B8B4A8BF90184918F3F21F418821B8A51
:107350001A8A21C04F5F5F4F5B8B4A8B4150504070
:10736000FA016491E82FF0E0EE0FFF1FE856FD4FA1
:107370000190F081E02D8F2D0995EA89FB893196E6
:10738000FB8BEA8B3197E491ED871E869E858D8578
:10739000981709F4B0CF8E858F5F8E8789858823F3
:1073A00019F420E030E047C08F858F3F11F08F5FE8
:1073B0008F879E819923C9F12F812223B1F18D817D
:1073C000882399F1899FC001112480509F4F892FF4
:1073D000992730E0AC01429FC001439F900D529F1E
:1073E000900D112480509F4F292F33278B818823A4
:1073F000F1F0EA81F0E0E050F148E491E058E89FD4
:10740000C001112480509F4F892F9927F601E81B56
:10741000F90BE29FC001E39F900DF29F900D1124A4
:1074200080509F4F292F332702C020E030E08A810F
:107430009C81890F8A83F8012083F3940A5F1F4F90
:107440006596F4E0FF1609F047CFDF91CF911F91C9
:107450000F91FF90DF90CF9008951F93CF93DF930C
:10746000582F90E0880F991F2091070E3091080E39
:10747000280F391FF90185919491DC011196FC01C7
:107480008491813011F413E01DC08091C70D8823D1
:10749000B1F08091D20D851711F4442381F48091CD
:1074A000DC0D882371F08091E70D851711F44423DA
:1074B00041F49091D60D8091EB0D891710F411E0F5
:1074C00001C012E0212F30E0FD01449185E190E000
:1074D000289FE001299FD00D389FD00D1124CF5453
:1074E000D24F4E871196BC8BAB8B1F8680E58A836B
:1074F0006F838FEF888719861A8A188A21E02A8776
:10750000198A5C8729831C82133049F481E091E059
:107510009093AA0D8093A90D2093A80D08C060E553
:10752000812F0E94803D6989812F0E949F3DDF91BC
:10753000CF911F910895FF920F931F93082FF62E5E
:107540000E94803D10E085E190E0089FF001099FD6
:10755000F00D189FF00D1124EF54F24FF2821F919D
:107560000F91FF900895962F482F50E025E130E0CD
:10757000429FF001439FF00D529FF00D1124EF54F4
:10758000F24F6281691B62830E94803D0895482FFB
:1075900050E025E130E0429FF001439FF00D529F03
:1075A000F00D1124EF54F24F9281690F62830E9413
:1075B000803D08951F93CF93DF93FA015491319644
:1075C0001491C52FD0E09F012F5F3F4F70E095E0F1
:1075D000660F771F9A95E1F7680F711D40E00BC0A9
:1075E00084918D939F5F31969517D0F34F5F2C0F49
:1075F0003D1F605E7F4F411730F4DB01A054BD4F4B
:10760000F90190E0F1CFDF91CF911F910895803C77
:1076100088F4282F30E0220F331FC90180519B4C82
:10762000FC0184912F503B4CF901949180935E0BA7
:1076300090935D0B60935F0B0895CF92DF92EF9272
:10764000FF921F93CF93DF938091200787FF0AC09B
:1076500090E08F709070009729F00196880F880F46
:10766000880F01C088E0E3EBF7E0108211821282FC
:10767000138234969AE0E33FF907B9F7C6EFDAE0F0
:1076800061E0C82EDD2419819881812F8150873DCA
:1076900008F055C0992309F452C09A3808F04FC039
:1076A000712F785040E050E0E12EFF24942F9A0192
:1076B0002E0D3F1D2C153D05E4F1283D3105CCF57F
:1076C000272F30E0D901AA0FBB1FAA0FBB1FAD5453
:1076D000B84F8C91882331F49295990F907E960F34
:1076E0009C9327C011968C911197882339F4929519
:1076F000990F907E960F11969C931BC0F901EE0F87
:10770000FF1FEE0FFF1FEB54F84F8081882331F4E9
:107710009295990F907E960F90830BC013968C9143
:107720001397882331F49295990F907E960F1396B4
:107730009C934F5F5F4F7F5F711709F0B7CF6F5F0B
:107740002396603209F09FCFDF91CF911F91FF9078
:10775000EF90DF90CF9008958F929F92AF92BF925B
:10776000CF92DF92EF92FF920F931F93CF93DF930D
:10777000882E962E5A016901F02E00E010E080EE6E
:10778000F80E0CC04F2D6E2D882D8C0F0E94703579
:107790002196CA15DB05B4F30F5F1F4F0C151D05AD
:1077A0002CF4C0E0D0E0E02EE90CF3CFDF91CF91D4
:1077B0001F910F91FF90EF90DF90CF90BF90AF900F
:1077C0009F908F90089540520E9470350895FF92C7
:1077D0000F931F93CF93DF938C01F62EEA01FE01E6
:1077E00044912196442349F0802F0F5F1F4F4F771C
:1077F00040526F2D0E947035F2CFDF91CF911F91D3
:107800000F91FF900895FF920F931F93182F062F4B
:10781000F42E42954F704A3010F4405F01C0495E2B
:10782000602F812F0E9470354F2D4F70812F8F5FF9
:107830004A3010F4405F01C0495E602F0E947035ED
:107840001F910F91FF900895FF920F931F93F82EB1
:10785000162F042F452F0E94033C402F612F8F2DA0
:107860008E5F0E94033C1F910F91FF900895EF924D
:10787000FF920F931F93F62E042F182FF8E0EF2E90
:10788000E80E07FF02C041E101C040E16F2D812FEA
:107890000E9470351F5F1E1511F0000FF2CF1F916F
:1078A0000F91FF90EF900895FF920F931F93CF9346
:1078B000DF93F62E042FEC0110E0002311F41123C6
:1078C00039F4802F6AE00E946145905F492F01C022
:1078D00040E06F2D8C2F0E9470351F5F2197133071
:1078E00031F0802F6AE00E946145082FE6CFDF91DA
:1078F000CF911F910F91FF900895CF92DF92EF9259
:10790000FF920F931F93CF93DF93C62E79018A01C5
:10791000EC01DD24E114F1040105110511F4DD2071
:1079200059F4C801B7012AE030E040E050E00E947D
:107930008045462F405F01C040E06C2D8C2F0E9497
:107940007035D394219786E0D81669F0C801B70145
:107950002AE030E040E050E00E948045C901DA01B1
:107960007C018D01D7CFDF91CF911F910F91FF90B7
:10797000EF90DF90CF9008957F928F929F92AF9279
:10798000BF92CF92DF92EF92FF920F931F93CF930C
:10799000DF93782E862E5A016901780100E010E00D
:1079A0000CC0A701692D872D8C0F0E94623521968E
:1079B000CA15DB05B4F30F5F1F4F0C151D052CF422
:1079C000C0E0D0E0902E980CF3CFDF91CF911F91C3
:1079D0000F91FF90EF90DF90CF90BF90AF909F906E
:1079E0008F907F9008957F928F929F92AF92BF92D7
:1079F000CF92DF92EF92FF920F931F93CF93DF937B
:107A0000782E862EEA01FA01C590D490FA013296BA
:107A1000A590B49000E016C0FC01EE0DFF1D32965B
:107A2000EE0FFF1FEC0FFD1F45915491692D812F23
:107A3000870D0E9462351F5F812F90E08C159D0598
:107A40005CF30F5F802F90E08A159B055CF48C9DA2
:107A500070018D9DF00C9C9DF00C112410E0902E77
:107A6000980CEACFDF91CF911F910F91FF90EF908B
:107A7000DF90CF90BF90AF909F908F907F900895B0
:107A80000F931F93CF93DF938C01C0E0D0E007C02A
:107A90000E94DA358823E1F30E94DD352196C01774
:107AA000D107B4F3DF91CF911F910F91089500009A
:107AB00000000000000000000000000000000000C6
:107AC00000000000000000000000000000000000B6
:107AD00000000000000000000000000000000000A6
:107AE0000000000000000000000000000000000096
:107AF0000000000000000000000000000000000086
:107B000099277727833008F00895E0E0F9E8660FB9
:107B1000771FE60FF71FA591B491E5E9FDE026E098
:107B2000289FE00DF11DA183B28311240895909147
:107B3000A80D9170880F892B8093A80D089599271F
:107B40007727E5E9FDE026E0289FE00DF11D6E3F77
:107B500031F46091A80D6E7F6093A80D0BC06F3F4C
:107B600031F46091A80D6E6F6093A80D03C07FE79C
:107B7000760F75831124089599277727E5E9FDE0AD
:107B800026E0289FE00DF11D6083112408952F93B6
:107B90003F934F935F936F937F938F939F93AF9395
:107BA000BF93789411240E941D3B0E9456340E947A
:107BB00047382F923F924F925F926F927F928F92AF
:107BC0009F92AF92BF92CF92DF92EF92FF920F936C
:107BD0001F93CF93DF930090920D002019F4A6E835
:107BE000BBE002C0ABE8BCE001E000260092920DD1
:107BF00002E00093930D2090960D3090970D4090E9
:107C0000990D50909A0D6090980D1091950D70906F
:107C10009C0D80909D0D90909E0DA0909F0DB0901A
:107C2000A00D20919B0DC090A20DD090A30DE090CF
:107C3000A50DF090A60D0091A40D3091A10D5091CD
:107C4000A70D6091A90D7091AA0D8091AB0D9FEFCA
:107C5000620C431CF2014491410300240008C12D31
:107C6000D02D970CA81CF501449142030024000874
:107C7000C10DD01D0C0DED1CF701449143030024F0
:107C80000008C10DD01D8A956AF44091A80D842F7B
:107C90008695062E0694062600FA7695679576F95F
:107CA00040FF66F940E860FD4FE745030024000807
:107CB000C10DD01DD595C7950024C038D0050CF056
:107CC000CFE70A94C038D0050CF4C0E8CD939A955C
:107CD00009F0BECF4091930D4A954093930D96E0E5
:107CE00009F0B6CF6092980D4092990D90929E0D3A
:107CF000A0929F0D0093A40DE092A50D6093A90D95
:107D00007093AA0D8093AB0DDF91CF911F910F91CE
:107D1000FF90EF90DF90CF90BF90AF909F908F90AB
:107D20007F906F905F904F903F902F909927809118
:107D3000600B77276091610B11240E947037BF910F
:107D4000AF919F918F917F916F915F914F913F91F3
:107D50002F910895A6E8BBE08AE092E000E00D9341
:107D60000197E9F7A6E8BBE0A093900DB093910DC1
:107D700000270093920D6FE760939A0D6093A00D1A
:107D80006093A60D61E06093A90D6093AA0D61E078
:107D90006093A80D66276093950D60939B0D60938B
:107DA000A10D6093A70D6093960D6093970D60935E
:107DB000980D6093990D60939C0D60939D0D609359
:107DC0009E0D60939F0D6093A20D6093A30D609331
:107DD000A40D6093A50D11240895E091900DF091EC
:107DE000910D019100580093B3000DE0E039F007C8
:107DF00006E81BE008F0F801E093900DF093910D78
:107E000008950C94033F0C94053F0F931F932ABDD4
:107E1000E091900DF091910D019100580093B30005
:107E20000DE0E039F00710F40000000010F0E6E883
:107E3000FBE0E093900DF093910DC895C895C8951F
:107E4000C895C895C8950000000000002AB51F918C
:107E50000F9108950000E091610BE0FFD6CFE1E1C2
:107E6000EA95F1F70000000008950000000000000E
:107E70000000000000000000000000000000000002
:107E800000000000000000000000000000000000F2
:107E900000000000000000000000000000000000E2
:107EA00000000000000000000000000000000000D2
:107EB00000000000000000000000000000000000C2
:107EC00000000000000000000000000000000000B2
:107ED00000000000000000000000000000000000A2
:107EE0000000000000000000000000000000000092
:107EF0000000000000000000000000000000000082
:107F0000000306090C101316191C1F2225282B2EFE
:107F1000313336393C3F414447494C4E5153555813
:107F20005A5C5E60626466686A6B6D6F70717374D0
:107F3000757678797A7A7B7C7D7D7E7E7E7F7F7F89
:107F40007F7F7F7F7E7E7E7D7D7C7B7A7A7978766F
:107F500075747371706F6D6B6A68666462605E5C85
:107F60005A585553514E4C494744413F3C3936339A
:107F7000312E2B2825221F1C191613100C0906035D
:107F800000FDFAF7F4F0EDEAE7E4E1DEDBD8D5D264
:107F9000CFCDCAC7C4C1BFBCB9B7B4B2AFADABA82F
:107FA000A6A4A2A09E9C9A9896959391908F8D8C52
:107FB0008B8A888786868584838382828281818179
:107FC0008181818182828283838485868687888A73
:107FD0008B8C8D8F9091939596989A9C9EA0A2A43D
:107FE000A6A8ABADAFB2B4B7B9BCBFC1C4C7CACD08
:107FF000CFD2D5D8DBDEE1E4E7EAEDF0F4F7FAFD25
:10800000808182838485868788898A8B8C8D8E8FF8
:10801000909192939495969798999A9B9C9D9E9FE8
:10802000A0A1A2A3A4A5A6A7A8A9AAABACADAEAFD8
:10803000B0B1B2B3B4B5B6B7B8B9BABBBCBDBEBFC8
:10804000C0C1C2C3C4C5C6C7C8C9CACBCCCDCECFB8
:10805000D0D1D2D3D4D5D6D7D8D9DADBDCDDDEDFA8
:10806000E0E1E2E3E4E5E6E7E8E9EAEBECEDEEEF98
:10807000F0F1F2F3F4F5F6F7F8F9FAFBFCFDFEFF88
:10808000000102030405060708090A0B0C0D0E0F78
:10809000101112131415161718191A1B1C1D1E1F68
:1080A000202122232425262728292A2B2C2D2E2F58
:1080B000303132333435363738393A3B3C3D3E3F48
:1080C000404142434445464748494A4B4C4D4E4F38
:1080D000505152535455565758595A5B5C5D5E5F28
:1080E000606162636465666768696A6B6C6D6E6F18
:1080F000707172737475767778797A7B7C7D7E7F08
:1081000000020406080A0C0E10121416181A1C1E7F
:1081100020222426282A2C2E30323436383A3C3E6F
:1081200040424446484A4C4E50525456585A5C5E5F
:1081300060626466686A6C6E70727476787A7C7E4F
:108140007F7D7B79777573716F6D6B69676563612F
:108150005F5D5B59575553514F4D4B49474543411F
:108160003F3D3B39373533312F2D2B29272523210F
:108170001F1D1B19171513110F0D0B0907050301FF
:10818000FFFDFBF9F7F5F3F1EFEDEBE9E7E5E3E1EF
:10819000DFDDDBD9D7D5D3D1CFCDCBC9C7C5C3C1DF
:1081A000BFBDBBB9B7B5B3B1AFADABA9A7A5A3A1CF
:1081B0009F9D9B99979593918F8D8B8987858381BF
:1081C00080828486888A8C8E90929496989A9C9EBF
:1081D000A0A2A4A6A8AAACAEB0B2B4B6B8BABCBEAF
:1081E000C0C2C4C6C8CACCCED0D2D4D6D8DADCDE9F
:1081F000E0E2E4E6E8EAECEEF0F2F4F6F8FAFCFE8F
:108200007F7F7F7F7F7F7F7F7F7F7F7F7F7F7F7F7E
:108210007F7F7F7F7F7F7F7F7F7F7F7F7F7F7F7F6E
:108220007F7F7F7F7F7F7F7F7F7F7F7F7F7F7F7F5E
:108230007F7F7F7F7F7F7F7F7F7F7F7F7F7F7F7F4E
:108500000309131E28313A40464C5054585B5E61B3
:10851000636567696B6C6E6F707172737475767773
:10852000777879797A7A7B7B7C7C7C7D7D7D7E7E99
:108530007E7E7F7F7F7F7F7F7F7F7F7F7F7F7F7F4D
:108540007F7F7F7F7F7F7F7F7F7F7F7F7F7E7E7E3E
:108550007E7D7D7D7C7C7C7B7B7A7A797978777770
:10856000767574737271706F6E6C6B696765636139
:108570005E5B5854504C46403A31281E13090300A4
:10858000C6CCD5DBDFE3E5E7E9EAEBECEDEEEFEFB8
:10859000F0F0F0F1F1F1F1F2F2F2F2F2F2F2F2F3C4
:1085A000F3F3F3F3F3F3F3F3F3F3F3F3F3F3F3F39B
:1085B000F3F3F3F3F3F3F3F3F3F3F3F3F3F3F3F38B
:1085C000F3F3F3F3F3F3F3F3F3F3F3F3F3F3F3F37B
:1085D000F3F3F3F3F3F3F3F3F3F3F3F3F3F3F3F36B
:1085E000F2F2F2F2F2F2F2F2F1F1F1F1F0F0F0EF78
:1085F000EFEEEDECEBEAE9E7E5E3DFDBD5CCC60037
:1086000000283D42302D2C2B2C2D2E2F303233358F
:1086100037393B3D3F414345484A4C4E50535557EF
:10862000595B5D5F61636567696B6C6E70717374D4
:10863000757778797A7B7C7D7D7E7E7F7F7F7F7F7B
:108640007F7F7F7F7F7F7E7E7D7D7C7B7A79787761
:1086500075747371706E6C6B69676563615F5D5B88
:1086600059575553504E4C4A484543413F3D3B397D
:1086700037353332302F2E2D2C2B2C2D30423D28E8
:1086800000E9E5FED4D7D7D7D6D4D2D0CECCCAC84D
:10869000C6C3C1BFBDBAB8B6B4B1AFADABA9A7A58B
:1086A000A3A19F9E9C9A999795949391908F8D8C5E
:1086B0008B8A89888887868585848484838383835D
:1086C0008383838383848484858586878888898A55
:1086D0008B8C8D8F909193949597999A9C9E9FA146
:1086E000A3A5A7A9ABADAFB1B4B6B8BABDBFC1C35E
:1086F000C6C8CACCCED0D2D4D6D7D7D7D4FEE5E917
:10870000F9F8F9F5EBE1DDDEE0E2E4E5E6E5E4E2E7
:10871000DED9D2CAC1B7ACA299918A868381808002
:108720008182838586888A8C8D8F90929395969787
:1087300098999A9B9B9C9D9D9D9E9E9E9F9F9F9F6F
:108740009F9F9F9E9E9E9D9D9D9C9B9B9A99989767
:1087500096959392908F8D8C8A888685838281806E
:10876000808183868A9199A2ACB7C1CAD2D9DEE250
:10877000E4E5E6E5E4E2E0DEDDE1EBF5F9F8F90059
:108780000708070B151F2322201E1C1B1A1B1C1E6B
:1087900022272E363F49545E676F767A7E7F7F7F31
:1087A0007F7E7D7B7A7876747371706E6D6B6A698B
:1087B0006867666565646463636262626161616182
:1087C000616161626262636363646565666768696B
:1087D0006A6B6D6E7071737476787A7B7D7E7F7F45
:1087E0007F7F7E7A766F675E54493F362E27221E42
:1087F0001C1B1A1B1C1E2022231F150B0708070019
:108800001F313D444E5354565A5F64696E747679F5
:108810007C7F7F7F7F7F7F7F7F7F7F7F7F7F7F7F6B
:108820007F7F7F7F7F7F7F7F7F7F7F7F7F7F7F7F58
:108830007F7F7F7F7F7F7F7F7F7F7F7F7F7F7F7F48
:108840007F7F7F7F7F7F7F7F7F7F7F7F7F7F7F7F38
:108850007F7F7F7F7F7F7F7F7F7F7F7F7F7F7F7F28
:108860007F7F7F7F7F7F7F7F7F7F7F7F7F7F7F7F18
:108870007F7F7F7F7F7F7F7F7F7F7F7C7871684C6A
:108880002C1C120C0A0B0A05FDF3E9DFD4CAC0B791
:10889000AEA69E97918B8685828080808080808026
:1088A00080808080808080808080808080808080C8
:1088B00080808080808080808080808080808080B8
:1088C00080808080808080808080808080808080A8
:1088D0008080808080808080808080808080808098
:1088E0008080808080808080808080808080808088
:1088F000808080808087919DACC4CBD4DDF2FAFA71
:1089000022002400260028002B002D003000330018
:10891000360039003D004000440048004C00510042
:1089200056005B00600066006C00730079008100F7
:10893000880090009900A200AC00B600C100CC00F5
:10894000D800E500F30001011001210132014401CA
:1089500057016C0181019801B001CA01E5010202D1
:108960002102410264028802AE02D70203033003EF
:1089700061039403CB03050442048304C704100578
:108980005D05AF0505066106C206290796070908B9
:10899000830805098E09200ABA0A5D0B0A0CC10C6E
:1089A000840D510E2B0F121007110A121D134014C3
:1089B0007415BA1614188319071BA31C571E2420FC
:1089C0000E22142439267F28E82A752D29300633F3
:1089D0000F364539AD3C49401B442848734CFE5086
:1089E000CF55EA5A51600C661D6C8B725A79928091
:1089F00037885090E598FDA19FABD3B5A3C0000088
:108A0000A0E0B0E0E6E0F5E40C94F845EC01A880C5
:108A1000B980CA80DB80A114B104C104D10441F43F
:108A200084E2A82E89EDB82E8BE5C82E87E0D82EDB
:108A3000C601B5012DE133EF41E050E00E94D5457C
:108A400027EA31E440E050E00E94B6457B018C010A
:108A5000C601B5012DE133EF41E050E00E94D5455C
:108A6000CA01B9012CEE34EF4FEF5FEF0E94B6451B
:108A70006E0D7F1D801F911F97FF04C061507040D5
:108A800080409048688379838A839B839B013F77EA
:108A9000C901CDB7DEB7EAE00C9414460E94004548
:108AA00008958EEA92E00E9400450895A0E0B0E0AB
:108AB0008093AE029093AF02A093B002B093B10244
:108AC0000895991B79E004C0991F961708F0961B2A
:108AD000881F7A95C9F78095089597FB092E072678
:108AE0000AD077FD04D02ED006D000201AF470955D
:108AF00061957F4F0895F6F7909581959F4F089562
:108B0000A1E21A2EAA1BBB1BFD010DC0AA1FBB1F91
:108B1000EE1FFF1FA217B307E407F50720F0A21B03
:108B2000B30BE40BF50B661F771F881F991F1A9470
:108B300069F760957095809590959B01AC01BD019A
:108B4000CF010895AA1BBB1B51E107C0AA1FBB1F81
:108B5000A617B70710F0A61BB70B881F991F5A95C9
:108B6000A9F780959095BC01CD010895629FD00131
:108B7000739FF001829FE00DF11D649FE00DF11DD8
:108B8000929FF00D839FF00D749FF00D659FF00D87
:108B90009927729FB00DE11DF91F639FB00DE11D74
:108BA000F91FBD01CF011124089597FB092E052659
:108BB0000ED057FD04D0A4DF0AD0001C38F4509525
:108BC0004095309521953F4F4F4F5F4F0895F6F7F1
:108BD00090958095709561957F4F8F4F9F4F089529
:108BE0002F923F924F925F926F927F928F929F92BD
:108BF000AF92BF92CF92DF92EF92FF920F931F93AB
:108C0000CF93DF93CDB7DEB7CA1BDB0B0FB6F8945B
:108C1000DEBF0FBECDBF09942A88398848885F849B
:108C20006E847D848C849B84AA84B984C884DF800C
:108C3000EE80FD800C811B81AA81B981CE0FD11DF0
:108C40000FB6F894DEBF0FBECDBFED010895F894C6
:028C5000FFCF54
:108C5200800080007F007D007B007800750071003D
:108C62006D00680062005C0056004F004800400042
:108C72003800300028001F0016000D000500FCFF20
:108C8200F3FFEAFFE1FFD9FFD0FFC8FFC0FFB9FF42
:108C9200B1FFAAFFA4FF9EFF99FF94FF8FFF8BFFF6
:108CA20088FF85FF83FF81FF80FF80FF80FF81FFB8
:108CB20083FF85FF88FF8BFF8FFF93FF98FF9EFF47
:108CC200A4FFAAFFB1FFB8FFC0FFC8FFD0FFD8FFC3
:108CD200E1FFE9FFF2FFFBFF04000D0016001F0099
:108CE200270030003800400047004F0055005C006C
:108CF200620067006C007100750078007B007D00E7
:108D02007F0080000000090012001B0023002C00DD
:108D120034003C0044004B00520059005F006500E3
:108D22006A006F00730077007A007C007E007F008B
:108D3200800080007F007E007C007A007700730054
:108D42006F006A0065005F00590052004B0044004A
:108D52003C0034002C0023001B001200090000001C
:108D6200F7FFEEFFE6FFDDFFD4FFCCFFC4FFBCFF41
:108D7200B5FFAEFFA7FFA1FF9BFF96FF91FF8DFFFF
:108D820089FF87FF84FF82FF81FF80FF80FF81FFD1
:108D920082FF84FF86FF89FF8DFF91FF96FF9BFF75
:108DA200A1FFA7FFADFFB4FFBCFFC4FFCCFFD4FF00
:108DB200DCFFE5FFEEFFF7FF20202020202020200F
:108DC20020202020202020202020202020202020A1
:108DD2002020202020202020202020202020202091
:108DE20020202020003CC3018A369836A837C73A93
:108DF200B33A9B36AA36B9369B3AC736D536010006
:028E020000006E
:00000001FF
